:020000040800F2
:10500000481C0020D5500008E98E00082D850008B6
:105010000000000000000000000000000000000090
:10502000000000000000000000000000519A00088D
:105030000000000000000000F19600088D9B0008B1
:10504000E7500008E7500008E7500008E750000864
:10505000E7500008255F0008E7500008E750000807
:1050600000000000E7500008015C0008E75000085D
:10507000E7500008D98A000800000000E750000847
:1050800000000000E75000080000000000000000E1
:10509000E750000800000000E7500008E750000853
:1050A000E7500008E7500008E750000801A6000894
:1050B000E7500008E7500008000000000000000072
:1050C0000348854600F0E8FC0048004775B9000831
:1050D000481C00200448804704480047FEE7FEE7DC
:1050E000FEE7FEE7FEE7FEE7299C0008C150000846
:1050F00030B50B46014600202022012409E00D4670
:10510000D5409D4205D31D469540491B25469540F7
:1051100040191546521E002DF1DC30BDF0B51FB40C
:105120000646002082B005464024019100901BE015
:10513000019922460F46304600F098FB049A059BE1
:10514000801A994110D310461946224600F07EFB82
:10515000361A8F410197224601200021009F00F05E
:1051600075FB38184D4100902046641E0028DFDC96
:10517000019B00982946324607B0F0BD03460B4319
:105180009B0703D009E008C9121F08C0042AFAD2FD
:1051900003E00B780370401C491C521EF9D2704783
:1051A000D2B201E00270401C491EFBD270470022BF
:1051B000F6E710B513460A4604461946FFF7F0FF16
:1051C000204610BD30B504460020034600E05B1CBD
:1051D000934203D2E05CCD5C401BF8D030BDF8B503
:1051E00002464A40D40F42004B0052085B089A42E4
:1051F00002D20246084611464A0023D0C30D4A0097
:10520000DDB2120EAD1A202D35DA49020126490A07
:10521000F6058A19002C00D0524220214F1B11465E
:10522000B9402A411018C20D9A4221D0002C17D043
:10523000012D08DCDA05801AD20F8019D207DBB203
:1052400000F040FBF8BDDA05801A012340001B0680
:10525000C01880185A428018CA0F1043490007E04E
:105260004908C2071143DA05801A801940088018DE
:1052700000F020FBF8BD61000122511A001BF7E786
:105280000122D2075140AAE70122D2075040A6E7E7
:1052900070B502464A40D50F40004A00ED0740086D
:1052A0005208002814D0002A12D0C40DD30D410298
:1052B0000120C0055202490A520AE41A09181218BC
:1052C0007D34914201D3641C00E04900002C01DAD6
:1052D000002070BD0023914201D3891A0343400886
:1052E00049000028F7D100290AD0914202D10121BA
:1052F000C90705E0914201D2012101E00121C94322
:10530000E005C018401900F0D5FA70BD420005D084
:105310004200120E52428A4201DB00207047C9054A
:1053200008187047F0B507460846584087B0C00FC8
:10533000049048000E46590040084908BC1A8841AC
:1053400005D2384631461E4617460B4602465800DF
:10535000400810434CD0300D039040055900400DDB
:10536000490D0590401A0290402872DA1803012175
:10537000000B09050843019004980092002805D00D
:1053800001995242002088410092019002984021E8
:105390000A1A0199009800F059FA05460C466B4626
:1053A00007CB00F074FAC0197141039A0E0D002367
:1053B000D71756401A467A40164344D0049A002A1A
:1053C0002DD0029A012A039A15DC1205C01A9141C8
:1053D00001263605001C7141D20F059ED2070093AD
:1053E000019202962A46234600F0B2FA07B0F0BDB9
:1053F00038463146FAE71605224A0F46B218C01A57
:10540000B74101210905001C4F4100187F41114699
:1054100018187941E20F10436D19644113E0E20757
:105420006D0815436408C2071443039A0126120548
:10543000C01A91413605001C7141CE074008304327
:105440004908C01851412A46234600F074FACDE7B6
:10545000FFE7049801224000C117121A00238B4174
:1054600004983146C417381AA141EEE730B401243C
:10547000E407634030BC55E730B40124E4076140E1
:1054800030BC4FE70000E0FFF0B51FB488B00B99C7
:105490000998002448400999C00F4900490809911A
:1054A000C0070B990090490049080B910999089889
:1054B000A64608431CD00B990A98084318D00998AF
:1054C00001244000420D4800410D099824050003C5
:1054D000000B204309900B980003000B20430B9016
:1054E00050181C494018002201901446104605E04F
:1054F000002001460DB0F0BD032801DA034600E0AC
:1055000003239C46C11A0AAE0AE05F0008ADED5BBA
:105510004F00F75B7D430027AA187C41491C5B1EA6
:105520006145F2DD410004AB5A522104120C0A43DA
:10553000240C401C0828DFDB01980290009970467B
:1055400001910090059B049A0799069800F000FAD3
:10555000D0E700000DFCFFFFF0B50C465C4085B0C5
:10556000E40FE40703944C000026640859009446B5
:10557000490802460296224321D062460A431ED0C1
:105580006200570D4A000E032303550D0124024605
:105590002C492405781B1B0B360B4018234326434C
:1055A000614600901C46501AB44103D30098401C39
:1055B000009002E0921800985B41002803DA002076
:1055C000014605B0F0BD00200121090507468646C9
:1055D00011E064461D46141BB54106D36546521BB7
:1055E000B341744607430C43A646CD07400849081B
:1055F000284392185B4105460D43EAD110461843F3
:1056000013D06046194650407140084306D06046AA
:10561000101AB34106D20122002306E00022012322
:10562000DB0702E00122D2435310009874460105C3
:10563000381C6141029C039D0019694100F07BF90F
:10564000BFE70000FD03000070B54B005B0803439B
:105650000BD04B005C0D002633466542B341D41796
:10566000AD1AA34102DB0020014670BD12053018BF
:10567000514170BDC217C10F504010B54018CA0744
:105680009623002100F01EF910BD10B500229623CC
:10569000114600F017F910BD0EB5C217C10F5040EA
:1056A000CA0740180021054B0293019200910A4657
:1056B0000B4600F04DF903B000BD000033040000BC
:1056C0000EB505490291002100910A460B46019151
:1056D00000F03EF903B000BD330400004100400279
:1056E0000122400AD205090E80187F2901DA002024
:1056F0007047962903DC9622511AC84070479639A4
:105700008840704770B5CD0F4A0009030123090B8B
:105710001B0519430B4BED070024520D9A4201DA89
:10572000002070BD074B34339A4203DC9A1A00F014
:105730009DF802E00449511888402C43F1D04042C2
:1057400070BD0000FF030000CDFBFFFF4A0009030E
:105750000123090B1B051943094B10B5520D9A4241
:1057600001DA002010BD064B34339A4203DC9A1A4A
:1057700000F07CF810BD03495118884010BD0000AE
:10578000FF030000CDFBFFFFC20FD207400040081F
:105790000BD0C10D0723DB01C91840020905400ADF
:1057A0001143C2084007114370470020014670476B
:1057B00010B5002904DB0124E40740428C41214656
:1057C000002B04DB1C460123DB075242A3418B4222
:1057D00000D1824210BD000010B5002904DB012475
:1057E000E40740428C412146002B04DB1C46012388
:1057F000DB075242A341994200D1904210BD000004
:10580000CB0FDB07490010B5490802460A4307D011
:105810000A0D07240903E401090B121B002A01DC0D
:10582000002010BDC900440F0C43C100E018D20590
:10583000801800F03FF810BD0122D207002800DBDD
:10584000101A002900DB511A8142704710B5202A36
:1058500004DB0146203A9140002010BD91402023F6
:105860009C1A0346E3401943904010BD10B5202A0E
:1058700004DB0846203AD040002110BD0B46D3403F
:10588000D0402024A21A91400843194610BD10B5FB
:10589000202A06DBCB170846203A1041C1170B43DC
:1058A00006E00B461341D0402024A21A9140084341
:1058B000194610BD002904DA401C490001D14008F6
:1058C0004000704770B40024050C05D1102400047A
:1058D00002D1002921D01124050E01D10002083483
:1058E000050F01D10001241D850F01D18000A41CEA
:1058F000002801DB4000641C002908D020252E1B55
:105900000D46F540A14000D001212943084301067E
:105910001B1B000ADB1D02D5002070BC7047DB0595
:10592000181880180029F8DA401C4900F5D170BC1D
:1059300040084000704710B5002B08DA0024401CD6
:10594000614192185B411A4301D14008400010BDEB
:10595000F0B51FB482B005460C0003D0084604F031
:1059600003FF02E004F000FF2030024600902146D1
:105970002846FFF76BFF049B059A04460F46184321
:105980001143084314D0184610431BD000984021FF
:105990000A1A18460599FFF769FF05460E46009A50
:1059A00005990498FFF752FF084305D0012004E051
:1059B0002046394607B0F0BD0020C11705430E430D
:1059C0002C43374300990E986305401A7905E40A81
:1059D00000220C43FD0A0A3002D500200146E9E707
:1059E0000105101969410C9C0D9D00196941FFF7D3
:1059F000A2FFDFE7FEB500231A461B1A8A4103DB2C
:105A00000020014603B0F0BD4A000D0301212D0B1B
:105A10000905520D0D43D10702D100186D41521EE8
:105A20005110FF31FF310131002704463E46384610
:105A3000009701910246012100200905FFF716FF9A
:105A4000C3197141F818324684468E464A41614670
:105A50002846611A904104D36046241A954176463F
:105A60001F46241900986D41401C00903428E1DD48
:105A7000F91930467041091BA84103D20022D243D4
:105A8000134601E00022134601980105381C7141BC
:105A9000FFF751FFB6E70000064C0125064E05E072
:105AA000E36807CC2B430C3C98471034B442F7D33F
:105AB000FFF70AFB60C8000880C8000870B58C18A2
:105AC0000578401C6B075B0F01D10378401C2A113D
:105AD00006D10278401C03E006780E70401C491C79
:105AE0005B1EF9D12B0705D40023521E0DD40B7079
:105AF000491CFAE70378401CCB1A921C03E01D787E
:105B00000D70491C5B1C521EF9D5A142D8D3002050
:105B100070BD000038B50446064805490068FFF727
:105B2000E7FA604300E0401E00900028FBD138BD3A
:105B300040420F005C010020F8B50446006881680F
:105B40008907890F012902D10168C90722D181681B
:105B5000114A10261140012500290ED181682943E0
:105B600081600120FFF7D6FF01F04EF907460CE0F7
:105B700001F04AF9C01B0A2807D9606D30436065FF
:105B8000A06D2843A0650120F8BD20680068C043CF
:105B9000C007EDD10020F8BD170000801FB50B48ED
:105BA00000900B4801900B4802900B480390694607
:105BB0000A4805F0CFF90A4A08481146083905F0A5
:105BC000B7F800F095FB002004B010BD6DC60008CA
:105BD00049C60008A9C60008A7C600086801002039
:105BE0001000002010B500231A4603E0845CE3187F
:105BF0009BB2521C8A42F9D3D84380B210BD000038
:105C000010B5034800F0BCFE024800F0B9FE10BD1C
:105C1000E8170020A017002030B5446C1C252C404C
:105C20000125A540046C6560046863608368102BDF
:105C3000036803D099600068C26030BD9A60006854
:105C4000C16030BDF0B58BB000200790864E0A20B1
:105C500005F030FD7D20400105F046FD834C844F6A
:105C6000E06B401CE06383480025089000226271CD
:105C70008148A18FC170090A017282740A214172A0
:105C80007E4909788172A18C0173457001467C4878
:105C9000103902784A75407888751C20002210312E
:105CA00005F0F2FD60790621484300211C3005F023
:105CB000FDFD022005F04EFD00210F2005F07AFCCD
:105CC00038422064F8D0206C411C18D040047DD5A7
:105CD0008122D20100210F2005F0ABFD0021102010
:105CE00005F068FC41066348490E0022C01D05F01E
:105CF00097FC6048C01D417A022902D09FE004F061
:105D0000A7FD5C4802225E490C30FFF75BFA0028D1
:105D10007ED105F01CFEE167A06705F005FE534A41
:105D2000803203C202900798039100281AD1012003
:105D30005049079053482139CB8E0380098F524A2E
:105D4000FF31C33189B2618491420BD95242891823
:105D500061845B1C4C4A99B20B320180914201D3A1
:105D6000002101800898444B6900027AC918099201
:105D7000CA74407A049008753E49684621394A8EB3
:105D80008280898EC1803B4904220831581CFFF76C
:105D9000F5F90198B04205DA064669460998087592
:105DA000049848753448032141724B220299D20469
:105DB00003980023891858410206080A10430190ED
:105DC00005F071FC01984108490000E04AE00A0E24
:105DD000080226498031CA6088602748E36F0A308C
:105DE000A26F05F089FD214880300CC822480E3092
:105DF00005F082FD1D488030C36882681E4812305D
:105E000005F07AFD00221C49192005F03DFD00E057
:105E100015E00021192005F049FD012005F09AFC4C
:105E20000006000E607305D100210F2005F0C2FBB3
:105E30000006F9D5802200210F2005F0FAFC6D1C28
:105E4000EDB20A2D00D211E70748864208D0002E95
:105E500006D00020A073022020706846808AE0846B
:105E60000BB0F0BD094AE6E7FFFF0100700000201B
:105E700000D02724E112002050140020240100202B
:105E80003801002044010020E7030000009027248F
:105E90001449012048720A4602205E3250720320E3
:105EA0003C3A507204200E3A50720F480D4B007865
:105EB000087022310870203108770C495A1C087884
:105EC00058714978997123331871597120331877B3
:105ED0005977107551751A461E3210755175107626
:105EE00051767047C01100201601002038010020B3
:105EF00010B503F083FD202003F03EFE012005F0E5
:105F000093FA002003F038FE044805F031F9044804
:105F100005F0E0FB002005F015FC10BD000100209D
:105F200083800000F8B503F035FE0520012100074D
:105F300000F056FF0025144C002800D06560134E79
:105F40000221304600F04CFF002815D101202070BE
:105F50000F48808F00280ED00127BF02002239464B
:105F6000304600F04AFF0A2004F052FE0122394672
:105F7000304600F042FF6560012000F069FE02201B
:105F800000F066FEF8BD000048010020000400504B
:105F9000C00D00207047000010B5084900224A617A
:105FA00007494B684C1523434B604B680824234337
:105FB0004B60C009C001026010BD00003018002015
:105FC000002002407FB500250C460646039500F0F0
:105FD0000FFEE009029003A901960095684600F0C3
:105FE0009FFD002804D000F0D7FD002004B070BD54
:105FF00000F0D2FD0120F9E710B5002302E0C45CF7
:10600000CC545B1C9342FAD310BD000010B5214A5A
:1060100000219069C305204804D541690223194332
:106020004161911593699B0505D54369012423437B
:1060300043616302194393695B0505D543690824ED
:1060400023434361E301194393691B0505D5436964
:106050000424234343616302194393699B0405D5D8
:1060600043691024234343616302194393699B03EB
:1060700004D5446920231C43446119439369DB031D
:1060800005D54369402423434361A0020143916144
:1060900010BD0000002002403018002070B50546F9
:1060A00000F0B2FE0646184C0AE0681C08D0002D2D
:1060B00004D000F0A9FE801BA84201D9032070BDC6
:1060C000A069C007F1D1A069800701D50220A061B5
:1060D000A069C00511D4A06980050ED4A06940054F
:1060E0000BD4A069000508D4A069800405D4A06978
:1060F000800302D4A069C00303D5FFF787FF012006
:1061000070BD002070BD000000200240F8B51746A9
:10611000002605460C4600F06BFD09E029460220EA
:10612000226800F047FD002804D1241D2D1D361DD6
:10613000BE42F3D300F030FDBE4201D20020F8BDD4
:106140000120F8BD10B5084902460020054B4979E9
:1061500005E044001C5B944203D0401CC0B288425E
:10616000F7D310BD641300207000002010B500F0BC
:106170003CFE10BD10B5094801F05CF880B2FFF795
:106180009FFA074A074BFFF77FF90022064BFFF7FC
:10619000E3F9FFF7DBFA80B210BD000054160020CF
:1061A000F853E3A59B843E4000408F4070B5002427
:1061B000204603F035FA47494748A200641CE4B280
:1061C0008150142CF9D3464944480A79027549791B
:1061D000417544490A780276497841763F4905205D
:1061E000133148720A2005F065FA7D20400105F060
:1061F0007BFA3A49002213310C2005F045FB0021BF
:106200000C2005F053FB384801F014F8344C0125FC
:10621000223C2085AD0309E0334801F00BF880B241
:106220002085E18EFF392D39884206DBE18E80B270
:106230008842F1D349198842EED8022005F08AFA43
:10624000002003F0EDF9294D00210F2005F0B2F9EF
:1062500028422064F8D0206C411C38D0400435D549
:106260008122D20100210F2005F0E3FA0021102045
:1062700005F0A0F941061948490E0022C73005F083
:10628000CFF9164DC735687A05281FD10222154966
:10629000681DFEF797FF002818D11148AE7C667183
:1062A0000422691C3630FEF769FF2946133108467F
:1062B00072000D466930FEF761FF607929464200A1
:1062C00005484838FEF75AFF0320207070BD04F0DF
:1062D000BFFA0000FFFF0100C413002021120020BC
:1062E00092000020380100205416002000D02724FE
:1062F00010B5144C1448224610321146083904F0E7
:1063000017FD0022114BE168A068FFF725F9104A3C
:10631000104B05F03BFC00220F4BFFF7ADF80022BD
:106320000E4BFFF7B1F8FFF76BFA2060002213461F
:10633000E168A068FFF73CFA01D0206810BD00209A
:10634000206010BD000000206801002000AA8F40DE
:106350006C45D9CC955BC83F0000F03F40A5E540B7
:1063600010B5084800F096FA0A21064800F032FA03
:10637000044800F01DF9800503D5024800F01AF921
:1063800080B210BDF8150020F8B52F4D0022012174
:10639000284600F032FDFFF7E3FFFFF776F92B4EBA
:1063A0003146FEF775FF2A4C0122A06011462846AF
:1063B00000F023FD2749A068002588423EDB2078B5
:1063C000254F002815D02570FFF7CAFFFFF75DF9AC
:1063D0003146FEF75DFFA060FFF7D6F900223B468D
:1063E000FFF744F800221D4BFFF74EF8FFF708FABD
:1063F0006060A068FFF7C8F900223B46FFF736F857
:10640000174A184BFFF740F806460F466068FFF73B
:10641000BBF9134A144B5242FFF736F832463B465B
:10642000FEF780FFFFF7ECF910496060884201DD5C
:10643000616004E0FF21C905C84200D3656060685F
:10644000FFF74CF9C0B2F8BD0004005000401B44F7
:10645000480000200000604000000C4000E0644064
:106460003333333333B33040CCCCEC3F0000C8423D
:10647000F8B5054604464035287C0026012808D09A
:1064800001202874206881688907890F01290ED1AD
:1064900001E00220F8BD0168C90708D0606D202125
:1064A000084360650126002028743046F8BD616D00
:1064B000FF2201329143022211436165C1688907BD
:1064C000890F0091C16889088900C16020688168CE
:1064D00092071143816000F097FC07460EE000F040
:1064E00093FCC01B0A2809D9606D02218843102142
:1064F00008436065002028740120F8BD206880688A
:106500000028ECDB2068C168009A1143C160606D0F
:1065100080088000401C6065C5E70000F8B50646AD
:106520000D464036317C01290DD0012131740168BE
:106530008A68520709D5416D202211434165002028
:1065400030740120F8BD0220F8BD174B6A68D805E9
:1065500047109A42154C8A6A2B6812D05B035B0B7A
:106560001A438A622968490305D5A1680143A160DD
:106570000A20FFF7CFFA2868800312D5A0683843B5
:106580000EE05B035B0B9A438A622968490302D5DC
:10659000A1688143A1602868800302D5A068B84340
:1065A000A06000203074F8BD0110000000270140F9
:1065B000406D70470068006C7047000070B50400C3
:1065C00006D0606D264600254036002802D006E041
:1065D000012070BDA5653574204600F0D3F8606DCC
:1065E000C00603D421688868400705D5606D102176
:1065F000084360653574EBE7606DFF22013290431C
:1066000002221043606588688207920F5B48012A66
:1066100002D10A68D2072BD1032362689B079A42F2
:1066200005D05B429A4202D05B009A4209D10A69C6
:10663000920092080A6121680A6963681A430A6134
:106640000CE00A69920092080A6181680F229204A4
:106650009143816081686268114381602168CA68E2
:1066600018239A43CA602168CA68A3681A43CA609B
:10667000816801225206914381608168A28E520690
:106680001143816020688168C90004D481680122B7
:106690001207114381602068C168394A1140C16006
:1066A0002069E168022825D00020014320462030DF
:1066B0000278037B52035B001A431143226B1143A0
:1066C000A26992031143E269D20311432268D3689D
:1066D0001943D160616A0A46FF3AC23A05D0A26AFC
:1066E00011432268D3681943D16042780121012AFD
:1066F00002D00BE00420D8E70078002823D0606D9A
:10670000202210436065A06D0843A065E06B01285E
:1067100020681FD00169C90703D0016949084900F1
:10672000016120684169C908C90041612068416967
:10673000A26B11434161A565606D80088000401C1B
:106740006065002070BD2068C26801231B041A43E5
:10675000C260DBE70269FF239B009A430261206865
:106760000269236CA66C1A43636C33431A430261BB
:10677000206802690A430261D3E700000027014054
:106780001902FEFF10B586B0044614216846FEF7D4
:106790000EFD0E492068884216D10D48416B421506
:1067A00011434163C16A01221143C162C06A694653
:1067B00010400590022000900320019000200290DC
:1067C0000520000700F050FA06B010BD002401407B
:1067D00000100240F8B504464069254640350E4693
:1067E00008280BD02068C068C00709D0606D202140
:1067F00008436065002028740120F8BD082700E0E8
:106800000C2700F001FB009011E0701C0FD0002E4F
:1068100005D000F0F9FA0099401AB04207D9606D2E
:10682000042108436065002028740320F8BD206817
:1068300000683842E9D0606D012149020843606573
:106840002068C16809058A0F0C21002A1BD120226B
:10685000125D002A17D10268120714D58268530707
:106860000122002B08DB43688B434360606D1302F9
:1068700098431043606506E0606D2023184360650F
:10688000A06D1043A065A069002801D120680160B7
:106890000020F8BD70B504462168002089684907CA
:1068A00021D425464035297C01291CD00121297499
:1068B000E169012904D02046FFF73EF9002811D1F3
:1068C000616D0A4A1140FF220132114361650021C6
:1068D000A165297422681C21116021688A6804233B
:1068E0001A438A6070BD022070BD0000FEF1FFFFF8
:1068F00030B5014620314A790023022A04D004220F
:10690000C2630B71012030BD026814680E25AC43D0
:10691000146002681468640864001460446C1C22EB
:10692000144001221546006CA54045604A71184686
:106930000B7130BD70B50024014620314A79022A1E
:1069400003D00421C163012418E0026813680E25F6
:10695000AB431360026813685B085B001360436C11
:106960001C221340012215469D40036C5D604A7154
:1069700000220A71816B002900D08847204670BD33
:10698000F0B4016C0D6801680C68466C1C2304228D
:106990001E401746B7402F420ED067070CD50C6833
:1069A000A40602D40C6894430C60416C19408A40E0
:1069B000016C4A60016B1AE00227B74002462F4083
:1069C0002032002F17D0A70715D50C68A40605D4D0
:1069D0000C680A25AC430C6001215171446C022102
:1069E0001C40036CA140596000211171C16A00294B
:1069F00018D0F0BC08470827B7402F4212D0240710
:106A000010D50C680E25AC430C60446C01211C4071
:106A10000B46A340046C6360C16351710021117186
:106A2000416BE4E7F0BC704770B504003CD01F48F0
:106A3000256814212818FEF75BFB800060641C4861
:106A400020640221204620300246417129681948FD
:106A5000E3680140A068666918432369334318431B
:106A6000A3691843E3691843236A1843084328605D
:106A70000121A0688903884210D00D488030836AC4
:106A8000656C1C210D400F26AE40B3438362656CDC
:106A900063680D40816AAB400B4383620020E06372
:106AA00001215171107170BD012070BDF8FFFDBF53
:106AB000000002400F80FFFFF8B504468C462030EE
:106AC00001790025012909D00126067141790027A5
:106AD000012905D0077102252846F8BD0220F8BD1E
:106AE00002214171E763206801684908490001609B
:106AF00061462046FFF790F8206B00282068016867
:106B000001D00E2205E00422914301602068016853
:106B10000A22114301602068016831430160DBE70C
:106B2000F8B51A4E0546307C0F46012807D00120E3
:106B300030741748FFF7B2FA010002D021E00220BA
:106B4000F8BD0020C04338606C6814E02046FFF7B1
:106B500023FA0F48FFF7A2FA01460E4842680823BD
:106B60009A434260426843159A434260002901D02B
:106B70003C6006E08034A8686A68C0018018A042C2
:106B8000E4D8002030740846F8BD0000301800201A
:106B900050C3000000200240054841680222114312
:106BA00041604168012211434160002070470000AC
:106BB00000200240F8B50C4C1646207C0F460128F8
:106BC00008D0012020740948FFF768FA0025002842
:106BD00002D006E00220F8BD65613E600348FFF781
:106BE0005DFA2574F8BD00003018002050C3000085
:106BF00011484168C9070BD0EFF3108172B60F4AF4
:106C0000C2600F4AC26081F310884168C9070ED183
:106C1000416889070DD5EFF3108172B6094A026108
:106C2000094A026181F310884068800701D501207C
:106C3000704700207047000000200240EFCDAB8974
:106C400005040302BFAE9D8C161514137047000097
:106C500010B504494A69024202D04861FFF7F6FFC5
:106C600010BD000000040140FCB500230124A2E097
:106C700027462A469F403A406FD04D68012D05D0E7
:106C8000022D03D0112D01D0122D16D185680326B7
:106C9000AC465D00AE46AE406546B543AC46CE68F8
:106CA0007546AE4065462E43866046680D79BE4304
:106CB000ED06ED0F9D4035434560C6685F00032536
:106CC000BD40AE46AE4335468E68BE402E43C660DC
:106CD0004E68022E01D0122E14D1DE08B6003618EE
:106CE0000196366A5D07B446EE0E0F25B540009654
:106CF0006646AE43B4460D69009EB54066462E43D7
:106D0000019D2E6206687546AE430D79AD07AD0F45
:106D1000BD40354305604D68ED004BD5294D6E6B88
:106D200026436E639E08284DB6007519AC46AD68C3
:106D30009E07360F0F27B740BD4305273F07B842D0
:106D400001D1002715E0214FB84201D1012710E001
:106D50001F4FB84202D102270BE02BE01D4FB84273
:106D600001D1032705E01C4FB84201D1052700E0FF
:106D70000627B7402F436546AF60184D2E684F6811
:106D80009643FF0300D516432E606E684F68964306
:106D9000BF0300D516436E60AE684F689643FF028E
:106DA00000D51643AE60EE684F689643BF0200D52B
:106DB0001643EE605B1C0A681546DA4000D057E7C0
:106DC000FCBD000000100240000001400004005023
:106DD00000080050000C0050001C0050000401404E
:106DE0000069084000D001207047426913460B40FB
:106DF0001B0491430B4383617047002A01D08161DA
:106E00007047816270470000014880687047000049
:106E1000500100200248816802788918816070471B
:106E20005001002010B50848002401684022114399
:106E30000160204600F00AF8002801D0012401E09A
:106E400000F042FA204610BD0020024070B5044612
:106E50000D4D7D202978C000FEF74AF901460B4808
:106E60000068FEF745F900F02BFF002809D1042C3B
:106E700007D200222146401E00F04EFA00206C602E
:106E800070BD012070BD0000500100205C01002099
:106E900070477047F8B502F07DFE604C0120E0704D
:106EA000208AFEF7F2FB01467F20C005FEF7F0F9CD
:106EB0005B4D06462968FEF792F928600120A16A19
:106EC000C005814201DA084603E03046FEF7DCF9EE
:106ED000A062FF21C9050025C84200D3A5626078E1
:106EE00000280BD102214F48FFF77AFF02004E49DC
:106EF0004E4817D00022FFF780FFE5620221494883
:106F0000FFF76EFF4A4E002855D0E562B08AFEF7C3
:106F1000BCFB434F3968FEF78FFC5FD24549012027
:106F200008705DE00122D1034048FFF766FF208A28
:106F3000FEF7ABFB01467F20C005FEF7A9F9E16A29
:106F4000FEF74DF93C49E0628842D7DD3848012719
:106F5000F926403000900A213046FEF7C9F8002992
:106F600003D131493148FFF701F902212D48FFF7DC
:106F700037FF002801D0002701E0002F12D10221A5
:106F80002848FFF72DFF00280CD104F0C7FD009919
:106F90000120888005F01EFB642003F039FE28499B
:106FA0002648C8600A2003F033FE3046761EF6B24B
:106FB0000028D0D1A2E7208AFEF767FB01467F2098
:106FC000C005FEF765F9E16AFEF709F91D49E062BF
:106FD00088429BDB1A491948C86097E71548057035
:106FE000708F401EFEF746FB3968FEF725FC06D879
:106FF0002079002803D014490120087001E01248CC
:107000000570708FFEF741FB3968FEF715FC04D25E
:107010002079002801D004F043FDF8BD14010020C0
:107020004C010020000400500080000000000050CF
:10703000C00D002076000020000040400400FA054A
:1070400000ED00E00000A04087000020704770B510
:10705000040010D0022025462035A873204601F0F8
:1070600043FDA87B032805D0204600F0B9F8002096
:10707000A873687370BD012070BD7047704710B56C
:10708000044600680168C943C90708D18168C9433B
:10709000C90704D1012141602046FFF7FBFE2068AB
:1070A0000168C943890708D48168C943890704D4A2
:1070B000022141602046FFF7EBFE20680168C943CA
:1070C000490708D48168C943490704D404214160B1
:1070D000204600F0F7F820680168C943090708D482
:1070E0008168C943090704D4082141602046FFF79D
:1070F000ADFF20680168C943C90608D48168C94347
:10710000C90604D4102141602046FFF7C2FE206862
:107110000168C943890608D48168C943890604D433
:10712000202141602046FFF7A9FF20680168C9437C
:10713000490608D48168C943490604D44021416006
:107140002046FFF79AFF10BDF8B5040005D025468C
:107150002035A87B002802D006E00120F8BD0020E1
:107160006873204600F04EF80220A8732068C268B9
:1071700084466368012B01D1062082431648616969
:10718000814202D0072040038243002B01D1D82046
:1071900082431248A668024018463043676A266A4E
:1071A0003E433043A66A30431043002B02D0012BEC
:1071B00004D005E02369E2691A4300E0E268104365
:1071C000054A914202D0A269114308436146C86052
:1071D0000120A8730020F8BDFFFF0000F8F119FF9F
:1071E00010B500680549884207D10548816B490000
:1071F000490881630D2000F073F810BD007C004049
:107200000010024010B50068084988420CD10848B7
:10721000816BC20411438163002201210D2000F023
:107220007BF80D2000F06CF810BD0000007C0040E1
:10723000001002400068C06970470000F8B50446BD
:107240000220254620351746A8731D480268C3044E
:107250001A4302602068C2689B121A43C260206809
:1072600002690126324302612268102050602068C2
:1072700081611021204601F0A7FC03281FD021685E
:1072800008204860206847610821204601F09CFCE6
:10729000032814D0204601F027FCA87B03280ED039
:1072A0002068816831438160206801693143016150
:1072B00020680169042211430161AE730020F8BD0A
:1072C00000040140704700000448416B0122114353
:1072D0004163816B020411438163704700100240D7
:1072E000002809DBC106C90E012088400349086057
:1072F000BFF34F8FBFF36F8F7047000080E100E056
:10730000002805DBC106C90E01208840014908603C
:107310007047000000E100E010B503F077FA10BDFF
:1073200002494A6882434A6070470000007000408A
:1073300002480168821511430160704700700040E7
:1073400002494A6802434A607047000000700040EA
:1073500005480168022211430160044801690422C2
:107360001143016130BF70470070004000ED00E044
:10737000F0B5154A1368154D54152D6A2340ED07D5
:10738000ED0F002B04D0002D02D01668A643166026
:107390001668B608B600064316600D48076904264D
:1073A0003743076101290DD040BF20BF20BF0169CD
:1073B000B1430161002B04D0002D02D0106820439E
:1073C0001060F0BD30BFF2E70070004000000140E7
:1073D00000ED00E0F8B5044600780027534D800624
:1073E00071D5524E403EB06BC00004D4B06BA905BD
:1073F0000843B06301274E480168C90511D40168EC
:10740000821511430160FFF7FFFC009005E0FFF7D4
:10741000FBFC0099401A642837D845480068C0052D
:10742000F5D532680321090560680A4001409142A0
:1074300008D08103890F032904D13168890301D55C
:107440000120F8BD2A69032109040A4022D008401E
:1074500090421FD0207880061CD528692A6988436D
:107460000121C9040A432A612A698A432A612861E1
:10747000C0050FD5FFF7C8FC009008E0FFF7C4FC7B
:107480000099411A2B48814201D90320F8BD28698F
:107490008005F3D561688803800F032805D1326821
:1074A0000005824301400A43326028690322616873
:1074B0001204114008432861002F04D0B16B012051
:1074C00000078143B1632078C00705D0E868A16850
:1074D000800880000843E8602078800705D5E868C8
:1074E0000C218843E1680843E8602078400706D50E
:1074F000E86803218902884321690843E86020780D
:10750000000706D5E8680321090388436169084339
:10751000E8602078000606D5E868032189048843DE
:10752000A1690843E8600020F8BD00004010024057
:107530000070004088130000F8B50E46050038D0F2
:107540005E480068C007C00FB04214D25B4C206890
:107550004008400030432060FFF756FC074605E036
:10756000FFF752FCC11B564881427AD82068C007F9
:10757000C00FB042F4D12878524C800705D5E0689E
:10758000F0218843A9680843E0602878C00752D0FA
:107590006868022806D0032807D0216801280AD08D
:1075A000890504E02168890301E021688901002937
:1075B00003DB0120F8BD4907F9E7E1688908890084
:1075C0000143E160FFF720FC0746686802280AD003
:1075D000032814D001281ED029E0FFF715FCC11B99
:1075E000374881423DD8E0680007800F0228F4D177
:1075F00021E0FFF709FCC11B3148814231D8E06826
:107600000007800F0328F4D115E0FFF7FDFBC11B35
:107610002B48814225D8E0680007800F0128F4D16B
:1076200009E0FFF7F1FBC11B2548814219D8E0684A
:107630000007800FF5D121480168C907C90FB14281
:1076400017D901684908490031430160FFF7DCFBA5
:10765000074608E005E0FFF7D7FBC11B1848814249
:1076600001D90320F8BD15480068C007C00FB0421B
:10767000F1D12878400706D5E06807210902884340
:10768000E9680843E0602878000707D5E06807212B
:10769000C90288432969C9000843E06000F03AF84C
:1076A000E168094A0906090F515CC84007490860AA
:1076B00007480068FFF7CAFBF8BD00000020024041
:1076C0008813000000100240AEC700085C010020D3
:1076D00054010020044805490068C968044A490566
:1076E000490F515CC84070475C0100200010024007
:1076F000C7C70008044805490068C968044A8904E6
:10770000490F515CC84070475C01002000100240E6
:10771000C7C7000870B51A4AD3681A490C20184028
:107720008D0004280CD04E00082810D00C2810D052
:1077300050680004410F0120C003491C884070BDFF
:107740001068C00601D5084670BD284670BD304699
:1077500070BD98020C4C000F205C1B029C0FD3687C
:10776000641CDB0301D5314603E01268D20600D465
:10777000294603F010F822460023FDF7CFFC70BD28
:107780000010024000093D00BEC70008FEB505001C
:107790007ED0FE4CE7680C20E6680740012000041C
:1077A00006402878C00747D0082F05D00C2F0AD1F3
:1077B00001200004864206D1206880033CD5686819
:1077C0000028E5D038E0012069680004814203D137
:1077D00021680143216011E0052301221B0492046A
:1077E0009942216802D111432160F1E78143216070
:1077F000216801400091206890432060686800285B
:107800000DD0FFF701FB009005E0FFF7FDFA0099AE
:10781000401A64287BD820688003F6D50CE0FFF777
:10782000F3FA009005E0FFF7EFFA0099401A642898
:10783000F0D820688003F6D42878800756D509232D
:10784000E868042F0DD00C2F01D1002E09D000289C
:107850003CD02168994301432160FFF7D5FA0646E1
:1078600028E02168490701D5002891D061681F22CE
:10787000120291432A6912021143616021689943FF
:1078800001432160FFF746FFE16809060A0F00E0A7
:107890008BE1BF49895CC840BE490860BE480068AA
:1078A000FFF7D4FA002873D120E0FFF7ADFA801B70
:1078B0000228AFD820684007F7D560681F21090269
:1078C000884329690902084360600FE02068400886
:1078D00040002060FFF798FA064604E0FFF794FAAC
:1078E000801B022896D820684007F7D42878C00665
:1078F00060D5002F0CD0A86900284AD02068FF214D
:10790000013108432060FFF77FFA06462EE0C1E010
:107910002068800502D5A8690028A6D060680721E4
:1079200049038843296A084360606068297F000230
:10793000000A090608436060286A410B0120C00361
:10794000491C8840E16809060A0F9149895CC840D2
:107950009049086090480068FFF778FA002817D12E
:1079600028E0FFF751FA801B0228A2D82068800582
:10797000F7D56068072149038843296A0843606096
:107980006068297F0002000A09060843606011E070
:10799000E2E02168FF20013081432160FFF734FAE3
:1079A000064604E0FFF730FA801B022872D82068F0
:1079B0008005F7D42878794E000724D56869002817
:1079C000306910D0012108433061FFF71DFA0090A3
:1079D00005E0FFF719FA0099401A02285AD83069D1
:1079E0008007F6D50FE0400840003061FFF70CFA41
:1079F000009005E0FFF708FA0099401A022849D8DC
:107A000030698007F6D42878400766D500200290B8
:107A1000A06BC00006D4A06B012109070843A06336
:107A2000012002905E480168C90511D401688215E1
:107A300011430160FFF7E8F9009005E0FFF7E4F972
:107A40000099401A642825D855480068C005F5D526
:107A5000FF20AA680130824203D1316901433161BC
:107A600011E001218902002A07D005231B029A4256
:107A700003D132690A433261EFE7326982433261EE
:107A8000306988433061A868002810D0FFF7BCF93E
:107A9000009008E05FE0FFF7B7F901460098091A87
:107AA0004048814257D830698005F4D50DE0FFF792
:107AB000ABF9009006E0FFF7A7F90099411A3948A1
:107AC000814248D830698005F5D40298002804D056
:107AD000A06B012109078843A063686A002866D06B
:107AE0000C2F3ED0012636060228206805D0B04370
:107AF0002060FFF789F905462FE0B0432060FFF7CB
:107B000083F9074604E0FFF77FF9C01B022822D85B
:107B100020688001F7D4E96AA86AE2680843296B03
:107B2000FD231B049A4311430843E060206830435F
:107B30002060FFF769F9054604E0FFF765F9401B8F
:107B4000022808D820688001F7D530E0FFF75CF9FB
:107B5000401B022801D90320FEBD20688001F5D416
:107B600025E00128F8D0E06801210904AA6A014053
:107B700091421AD10F218904EA6A0140914214D13D
:107B8000032189050840296B88420DE0001002405E
:107B9000AEC700085C0100205401002040100240E4
:107BA000007000408813000001D00120FEBD0020BD
:107BB000FEBDF8B504000ED0FF27606A053700252A
:107BC00000280AD02561656126464036A562707C92
:107BD000002807D00AE00120F8BD6068B842F3D061
:107BE000E561F1E73574204600F03EF8022171743A
:107BF0002068026840239A4302602123A2686068DB
:107C00009B021A4038401043E3688A02134018432D
:107C100023690B40217D1843C907C90F0843A16997
:107C2000931019400843E169382319400843216A39
:107C3000802319400843A16A930019400843216832
:107C40000860A0690421000C0840616A10231940F3
:107C50000843216848602068C1699143C161656536
:107C6000012070740020F8BD10B586B004461421C0
:107C70006846FDF79CFA10492068884219D10F48E0
:107C8000416B821411434163C16A01221143C162F5
:107C9000C06A002110400590E02000900220019071
:107CA0000320039002910491052069460007FEF726
:107CB000DBFF06B010BD00000030014000100240A4
:107CC000094910B5401E884201D9012010BD074C5A
:107CD00060610321081F02F099FD0020A0610720C8
:107CE0002061002010BD0000FFFFFF0000E000E069
:107CF000F0B502462032137E012B1ED001251576E9
:107D00000223537606687468B3687027BC430F6813
:107D1000274377600068AC07A04205D0084CA0421A
:107D200002D0084CA04204D180244968A3431943DF
:107D30008160557600201076F0BD0220F0BD000075
:107D4000000801400014014070B5050005D02C4624
:107D50002034607E002802D006E0012070BD0020A3
:107D60002076284600F010F802206076291D286849
:107D700001F086FF0120A077A076E076207760777B
:107D80006076002070BD00000068012189078842EC
:107D900004D10348816B01221143816370470000C5
:107DA00000100240F8B5054604462035287E01281B
:107DB00017D001262E7602206876226890687727F1
:107DC000FF23B8431B02984390600A68502A31D0C1
:107DD0000EDC202A4BD006DC002A48D0102A3AD1EB
:107DE00045E00220F8BD302A41D0402A33D136E0A8
:107DF000602A27D0702A12D001200003121A2AD03C
:107E0000824228D1CB684A688968206801F071FFF6
:107E10002068816801229203114381601BE0CB68D6
:107E20004A688968206801F064FF216888683843DF
:107E3000886010E0CA684968206801F0D4FF5021CA
:107E4000206806E0CA684968206801F0DDFF60210B
:107E5000206801F059FF6E7600202876F8BDCA68C8
:107E60004968206801F0BFFF40212068F1E7114612
:107E70002068EEE710B586B0044614216846FDF789
:107E800096F9012120688907884212D10A49CA6AF5
:107E900002200243CA62C96A019001400591410271
:107EA0000091002102910391049069460348FEF776
:107EB000DBFE06B010BD00000010024000040050C0
:107EC000F8B5064604462036307E0D4601280BD014
:107ED000012008273076002A08D0042A16D0082A64
:107EE0002AD00C2A4DD137E00220F8BD206801F0DD
:107EF00013FF206881693943816120688169042208
:107F00009143816120688169EA6812E0206801F08C
:107F10001BFF206881690122D20211438161206820
:107F20008269012189028A43826120688169EA6845
:107F300012021143816124E0206801F01EFF2068D5
:107F4000C1693943C1612068C16904229143C1619B
:107F50002068C169EA6812E0206801F029FF206802
:107F6000C1690122D2021143C1612068C2690121A5
:107F700089028A43C2612068C169EA68120211431A
:107F8000C16100203076F8BD70B5050005D02C46E3
:107F90002034607E002802D006E0012070BD002061
:107FA0002076284600F00FF802206076291D286808
:107FB00001F066FE0120A077A076E076207760775A
:107FC0006076002070BD704770B505462C460220D3
:107FD0002034002908D004290BD008290ED0627F54
:107FE000012A10D0012070BDA27E012AFAD1A0760C
:107FF0000AE0E27E012AF5D1E07605E0227F012A3F
:10800000F0D1207700E060770122286801F064FE5B
:108010000122286892070121904205D0074A904228
:1080200002D0074A904204D182685207520F062AB2
:1080300002D002680A430260002070BD00080140BF
:108040000014014070B504460D460068002201F09E
:1080500043FE2068016A0C4A114203D101684908B5
:108060004900016001202034002D06D0042D06D0E7
:10807000082D06D06077002070BDA076FBE7E07683
:10808000F9E72077F7E7000011110000704770470B
:1080900070470000F8B502680446D0691168966818
:1080A000814B05461D402023002D6CD0F7077F4DE6
:1080B000FF0FBC460D402F4379D02546C7078035BA
:1080C000002F06D0CF0504D5012717622A683A434E
:1080D0002A60820708D5F20706D0276802223A6292
:1080E0002A6804273A432A60420708D5F20706D0D7
:1080F0002668042232622A68022632432A60020776
:108100000AD50A461A406646324305D02668082238
:1081100032622E6816432E60020508D54A0106D544
:1081200001222668D20232622A681A432A602A682B
:10813000002A30D0800606D5880604D5616E002955
:1081400001D020468847286821688968490602D4FA
:108150002821084225D0204602F069F8206881686D
:10816000490619D5826840218A438260206F002821
:1081700012D04F498163206FFEF7DCFB00280AD044
:10818000206F816B06E0850611D58D060FD5616ED7
:1081900077E020468847F8BD2046FFF779FFF8BD15
:1081A00005E02046FFF774FF00202860F7E7256E02
:1081B000012D56D1C50654D5CD0652D510261662CE
:1081C0002068816825464906403500292ADA226F51
:1081D000116849680904090CE1D02F8B8F42DED960
:1081E000698311680968890617D4016832019143CF
:1081F00001602068816849084900816020688168C1
:10820000402291438160E367002020662068016876
:10821000B1430160206FFEF76BFB288B698B401A1E
:1082200081B21AE0298B6A8B891A6A8B89B2002A7B
:10823000B5D00029B3D00268FF252135AA430260DA
:1082400020688268520852008260E367002020663E
:10825000606620680268B24302602046FFF716FF9E
:108260009DE7C50208D5750206D5012000051062FC
:108270002046FFF70CFF92E7050605D50D0603D54E
:10828000A16E002985D18AE7400688D5480686D5A3
:10829000116820464024A143116083670021816654
:1082A00000F043F97BE700000F0800002001000404
:1082B00055A1000810B5040003D0A06F002802D01B
:1082C00007E0012010BD002174200155204600F078
:1082D00027F82420A0672068016849084900016048
:1082E000204601F0F7FF0128ECD0606A002802D098
:1082F000204601F019FE206841680922D20291430C
:108300004160206881682A22914381602068016869
:10831000012211430160204601F06CFE10BD0000F7
:10832000F0B587B0064614216846FCF740FF2C499B
:108330003068884251D12B48416B0122920311438E
:108340004163C16A01221143C162C06A0025104025
:1083500005900320400200900220032701A9A1C13B
:1083600004200490052069460007FEF77DFC1F4CA1
:108370001D48A560E56081C48027E560A7602020D6
:10838000256160610002A0611848083CFEF74CFBC3
:10839000002801D0FDF7FEFD3467A662144C124898
:1083A0002146143820600320606010200831A1C1EC
:1083B0006561A561E56120462562FEF735FB002871
:1083C00001D0FDF7E7FDF466002201211B20A66223
:1083D000FEF7A2FF1B20FEF793FF07B0F0BD0000E1
:1083E000003801400010024030000240A017002079
:1083F000E817002070B5C36F202B27D100290BD0C0
:10840000002A09D0012483682403A34206D103690A
:10841000002B03D1CB0701D0012070BD0346603390
:108420001C7D012C12D001241C7500230366084C0E
:108430000368A34207D05C68240204D51C680125A8
:10844000AD062C431C6002F045F870BD022070BDE3
:108450000048004070477047FFB50446806F83B006
:1084600017460D4620285ED1002D0AD0002F08D0D7
:10847000A168C001814207D12069002804D1E80722
:1084800002D0012007B0F0BD204660300090007D92
:10849000012848D000980121017500208021085151
:1084A0002120A067FEF7B0FC2646403601903782B7
:1084B00077820120A1680003814202D1206900284F
:1084C00005D02F46002500990020087511E00027EF
:1084D000F9E700228021204602F042F8002815D159
:1084E000002F15D02168387888627F1C708A401E62
:1084F0007082708A019B002806980090E9D10022C2
:108500004021204602F02CF8002808D00320B9E7CB
:1085100028882168C005C00D8862AD1CE6E72020D0
:10852000A0670020AEE70220ACE77047034D044C83
:1085300004A002F00FF9E560FAE700000400FA0574
:1085400000ED00E0486172644661756C745F4861DB
:108550006E646C65722E0D0A0000000000B585B0D7
:1085600014216846FCF723FE04490220C880044910
:10857000488300F053FC05B000BD0000000E002051
:108580001401002010B505242407002204212046F0
:10859000FEF733FC002208212046FEF72EFC0A20BD
:1085A00002F03DFB012204212046FEF726FC0A20B2
:1085B00002F035FB002204212046FEF71EFC10BD10
:1085C00010B505242407002204212046FEF715FCDF
:1085D000012208212046FEF710FC0A2002F01FFBB2
:1085E000012204212046FEF708FC0A2002F017FBB6
:1085F000002204212046FEF700FC10BDF8B500243F
:108600000526074625463607002204213046FEF798
:10861000F4FB0A2002F003FB012204213046FEF79E
:10862000ECFB6006040E08213046FEF7D9FB00285B
:1086300001D0641CE4B2052002F0F1FA6D1CEDB229
:10864000082DE1D3002F03D0FFF79CFF2046F8BD93
:10865000FFF7B6FFFAE770B5052605463607002294
:1086600004213046FEF7C9FB0024E80901D00122AD
:1086700000E0002208213046FEF7BFFB6806050E29
:108680000A2002F0CCFA012204213046FEF7B5FBA5
:108690000A2002F0C4FA002204213046FEF7ADFBA6
:1086A0000A2002F0BCFA641CE4B2082CDDD370BDD1
:1086B00010B505242407012208212046FEF79DFB62
:1086C000012204212046FEF798FB002208212046C3
:1086D000FEF793FB0A2002F0A2FA002204212046B2
:1086E000FEF78BFB10BD10B50524240700220421E2
:1086F0002046FEF782FB002208212046FEF77DFB84
:108700000A2002F08CFA012204212046FEF775FBB4
:10871000012208212046FEF770FB0A2002F07FFAB2
:1087200010BD70B505252D0700240122082128461B
:10873000FEF763FB062002F072FA012204212846AC
:10874000FEF75BFB062002F06AFA07E0641CE4B265
:10875000FA2C03D9FFF7C7FF012070BD0821284676
:10876000FEF73EFB0028F1D1002204212846FEF747
:1087700044FB002070BD0000F8B501F06DFC01F075
:108780009DFC5B480068C069FDF7F4FC594C5A49F0
:10879000A082898F594E0025002931D0A26A730327
:1087A00057499A4202DB02220A7000E00D700A78F3
:1087B00001218902002A05D0012A0ED0022A10D0F8
:1087C000032A1DD1608B01282ED0022818D14848D9
:1087D00008214038FFF736FC12E0FF22F5329042C4
:1087E000F0D2608B01281DD0022804D008E030466A
:1087F000FEF703FB04E03E4808214038FFF7E4FBA6
:10880000FDF7C2FD20700121C9023046FEF7E8FAEB
:108810000127FF0300282DD03A480560A0790028E1
:1088200004D007E00022E2E70122E0E70120A07186
:1088300001F0F8FE80213046FEF7D2FA002806D07B
:10884000002208213046FEF7D8FA012205E0012275
:1088500008213046FEF7D1FA0022052039460007EC
:10886000FEF7CBFA244C284E4034A08C274F012829
:1088700003D01CE0A5710022EAE72548694608807C
:1088800072B680212348FDF79DFB002804D0022208
:1088900069462048FDF73AFC62B61FA001F05AFF76
:1088A000A58403F097FE642002F0B2F9FE60608CAC
:1088B000012808D110486584058003F08BFE6420F0
:1088C00002F0A6F9FE60208C012806D1258403F071
:1088D00081FE642002F09CF9FE600748124A01887C
:1088E000914202D1C088002800D1FE60F8BD00008E
:1088F0001C17002014010020C00D002000040050AF
:10890000850000204C0100200400FA0500ED00E085
:10891000AAAA0000384A0008BDF8C8EBC9FDBCB6D9
:10892000C4A3CABD0D0A0000AA55000038B5002432
:108930006946202000F0AAF868460078572800D041
:1089400001246946212000F0A1F868460078032838
:1089500000D001246946222000F098F8684600788B
:10896000402800D001246946232000F08FF8684693
:108970000078082800D001246946302000F086F8ED
:1089800068460078AA2800D001246946322000F009
:108990007DF80C486946008F0978884200D0012490
:1089A0006946332000F072F8064869464030408836
:1089B0000978884201D1002C02D004490248C860DD
:1089C00038BD0000C00D00200400FA0500ED00E0F5
:1089D00038B55721202000F07AF80321212000F03B
:1089E00076F84021222000F072F80821232000F0C0
:1089F0006EF8AA21302000F06AF81048018F14297F
:108A000001D8002901D1012101870C4C4034618833
:108A1000142901D8002901D102216180008FC1B23F
:108A2000322000F054F8A178332000F050F8684666
:108A300000F006F80A2002F0F2F838BDC00D002060
:108A400010B501460F2000F021F8002800D00120C9
:108A500010BD10B50446FFF72BFE3220FFF7FBFDDB
:108A6000FFF75FFEE0B2FFF7F6FDFFF75AFEFFF7F4
:108A70001FFE3320FFF7EFFDFFF753FE0020FFF747
:108A8000BDFD0446FFF72FFE204610BD10B50C4675
:108A9000FFF7DFFF2070012010BD70B50D460446C2
:108AA000FFF706FE3220FFF7D6FDFFF73AFEE0B2F1
:108AB000FFF7D1FDFFF735FE2846FFF7CCFDFFF7A6
:108AC00030FEFFF710FE0A2002F0A9F870BD10B5C5
:108AD000FFF7E3FF012010BD10B50248FEF7CFFA03
:108AE00010BD000054160020FEB50446002772B6E3
:108AF000334A01688B1804D13248C76803208004C8
:108B0000074088680190C868009048698E69002B0A
:108B100008D12C4940398B6ACD042B438B628B6A78
:108B2000AB438B62014631433CD025492368CB429D
:108B300005D12449CA6803239B049A43CA60254689
:108B40002035002810D021680A6901231A430A61E0
:108B5000216848610821204600F036F8032800D13A
:108B6000A873216808204860002E10D02068016991
:108B7000012211430161206886611021204600F026
:108B800023F8032800D1A8732168102048600C48FE
:108B90002168C14206D10B48C16803229204914367
:108BA0003943C160206801694908490001612168B1
:108BB0000198886021680098C86062B6FEBD000018
:108BC0000084FFBF4010024070B506460B480D46BA
:108BD000002409490068FCF78BFA7D21C90048434D
:108BE0003168401E00D103240B682A469A4301D005
:108BF0000028F6D1204670BD204E00005C01002008
:108C00001CB5002116480091144A01910260C1630D
:108C100012054260816007228263012202610246DE
:108C2000C16020321170FF235170C23343628162F0
:108C3000117301638161042241634261C161FDF7E7
:108C4000BDFC084800908013019069460448FDF778
:108C500065FC00210248FDF70BFC1CBD002401400F
:108C6000F81500200200000408B50848016B012235
:108C700011430163006B01211040009000220A2083
:108C8000FEF74AFB0A20FEF73BFB08BD001002403E
:108C9000F0B587B014216846FCF789FA4748C26AE4
:108CA00004210A43C262C26A0A400592C16A802650
:108CB0003143C162C16A31400591C16A0124214337
:108CC000C162C16A21400591C16A02252943C1627E
:108CD000C06A22462840059005201C210007FEF7A7
:108CE0008CF8012236493748FEF787F800223649CA
:108CF0003448FEF782F8912105200022090200077E
:108D0000FEF77BF83148019000270520694602975D
:108D100000940007FDF7A8FF0C200090112001909F
:108D2000032003900520029769460007FDF79CFF8A
:108D300010206A46039591C2052069460007FDF799
:108D400093FF1120019002976946039700941D48F4
:108D5000FDF78AFF1E480190694600950294194864
:108D6000FDF782FFE00200906946019702951548E1
:108D7000FDF77AFF1748694691C169461148039784
:108D8000FDF772FF91200002694691C105206946F6
:108D900000070397FDF768FF69460A4801970096A8
:108DA0000294FDF761FF002201210520FEF7B4FACD
:108DB0000520FEF7A5FA07B0F0BD00000010024044
:108DC00001020000000400500830000000001110F3
:108DD000000021100832000010B50F4C0D48206033
:108DE000FF20053060600020A060E06020616061CD
:108DF000E0610121206249026062A161A062072056
:108E0000E0622046FEF7D5FE20680168402211434B
:108E1000016010BD003001408416002010B58AB0FA
:108E2000002404940594069407940894012118489A
:108E30000994009401940294890703940160092124
:108E400084604160046113494461C160FEF77CFFA6
:108E500001200003049004A90D48FEF7A3FF0C486D
:108E6000FFF792F8089408A909480994FEF740FF13
:108E700060200090084801900294082269460394FB
:108E80000348FFF71DF80248FEF7F4FF0AB010BDD3
:108E9000DC160020930400005702000000B585B0E6
:108EA00014216846FCF783F90E480D490160E12161
:108EB0004902416000218160C160016181610C2231
:108EC000C161426101623021416201210903816374
:108ED0004900C163FFF7EEF901F09EFB05B000BD4C
:108EE000003801401C17002070470000F0B589B021
:108EF0000A2002F0DFFB7D20400102F0F5FBFD4C73
:108F00000025A570FC482066A07C2F460C2801D3C4
:108F10000B20A07460790A2801D90A206071F748F3
:108F2000E570F74E00783071F649A0790978400075
:108F30000843E17D89000843F071E06BF070010A9D
:108F40003172401CE0636079B07442003046EE49F3
:108F50001330FCF713F96079EB4982004000801967
:108F600060311330121DFCF709F9607906214200C7
:108F700048438019E5491730921CFCF7FFF82E2072
:108F8000205E002803D0E249098A0818E08560794C
:108F9000D849C000223182190B7B53764B7B9376E4
:108FA00006227272DB4A1D301278B272A28C3273C2
:108FB000D34A0B79133A1375497951750022D04978
:108FC00002F062FC60790021C0001D3002F06EFCEE
:108FD000D148FEF72FF9208509E0CF48FEF72AF99E
:108FE00080B22085E18EFF392D39884208DBE18E81
:108FF00080B28842F1D30122920389188842ECD8CA
:10900000022002F0A7FBBE480126C571E574E57396
:1090100066742574C048FEF70DF960850290E5700E
:109020006079FCF74DFBBD4ABD4BFCF72DFA01F012
:109030008BFD0022BB4BFCF775F9FCF787FB0006A4
:10904000C10C0298081880B2F103A085884201D3B0
:10905000401AA085B448E0642079401C2071AE48D5
:10906000FEF7E8F82085A848A2496438403101910C
:109070000790C2E1A848FEF7DDF820850BE0A6487E
:10908000FEF7D8F880B22085A18D884203D3A74A85
:109090008918884207D300210F2002F08BFAA449D7
:1090A00020640842EBD0206C411C1FD040047DD5C9
:1090B0008122D20100210F2002F0BBFB00211020F1
:1090C00002F078FA41069048490E00227C38E165AA
:1090D00002F0A6FA002002F007FB002002F0B9FA25
:1090E00089487C38417A0729C3D101E001F0B0FBFF
:1090F00002229049401DFCF765F80028B9D102F022
:1091000026FCE167A06702F00FFC7A4B803303C3B3
:10911000E0787D49401CE07083390B7A6846037023
:10912000497A417000880490E18C88427ED174496C
:1091300081488C31C98E018071496E488C31098F0C
:1091400041847548FEF776F8208502F045F96948B4
:109150007D22803001684068D2040023891858417C
:109160000206080A10434108490000900A0E08024E
:1091700060498031CA6088606148E36F0A30A26F3D
:1091800002F0BAFB607981005D4808185949163031
:1091900080310CC902F0B0FB56488030C368826849
:1091A0005748123002F0A8FB082100E018E15448AB
:1091B0004172B430C07C0009A07514D0524802221C
:1091C0005C497738FBF7FEFF00280CD14C48E67469
:1091D000C671E06D4C491638C2B26639C81D227599
:1091E000FB30FBF7CBFF60790022800044491C3044
:1091F00002F04AFB6079002180001C3002F056FB2F
:10920000009802F050FA012002F0A4FA60730221E3
:109210004A48FDF7E5FD002824D000213948384AA6
:1092200001708C32518E0198049100E08AE0018136
:10923000918E41818C46D11DFD310A68A06C82421D
:1092400001D07F1CFFB2E06408602F4920657C39A3
:10925000C97C0907090F032900D06175E16D1C293C
:1092600002D016E00121D9E72549224A8C31C98F65
:109270001186264A079B183A1B881383884207DD0C
:10928000002805DD002903D0207E401C207600E068
:1092900025762571E6730198049981816146C18123
:1092A0002674608C2649FF30C33080B260848842C7
:1092B0000CD94942401860841F487D220188D200A1
:1092C000491C89B20180914200D305801A487D2152
:1092D0000088C9004843618C4018606500F0F6FBC7
:1092E000607B002805D100210F2002F063F9000601
:1092F000F9D58BE0700000203F420F0014010020E0
:1093000034120020480100206413002018150020AA
:10931000000E00202401002054160020B81E85EB0A
:1093200051B8CE3F00000840A0860100983A0000E6
:1093300000D0272438010020440100200004005000
:10934000E7030000FCF7FEFE724A03211154724B42
:1093500001995A8E0A819A8E4A81E16D22461C2912
:1093600005D16E4B4100CB180799098859808000C0
:109370006849694B6039009041189B8F0B806549A3
:10938000303941184B68906C834201D07F1CFFB28A
:109390004860614900988C394018614916300CC901
:1093A00002F0AAFA216EA06C884208DA594A0099A4
:1093B000603A5158012902D1206604990691554915
:1093C000009A60398958814217DD012915DD22464E
:1093D000002812DD0498D08402201070A5730CE0E0
:1093E000504A00210F2002F024FA6079E178401CF5
:1093F000814202D0002002F02CF9218DA08D814203
:1094000000D237E6484A80188142FAD8E07B01282A
:1094100001D00220E07301F0DFFF424A00210F205B
:1094200002F007FA2079002817D0404909888A00FD
:109430008A18824200D22670002000F0F1F8E07C09
:1094400000283AD033490C310B78A3724878607207
:109450008A782272022B17D02FE0E06C216E32380E
:1094600081420FDAE179314A491CC9B2E1711288AF
:10947000204652008A42E2D20699C184022101703C
:10948000A573DCE7E571DAE710280CD0C82814D200
:10949000274BC91C1818FBF771FE03F09BF86420DA
:1094A00001F0B6FB22E6234800684000000E04D11C
:1094B000C878FCF7EAF81F490860022F01D9E57265
:1094C00006E0E07A411CE172032801D9E5722670BA
:1094D00000202378A27B65790FE00E4E4100903E7C
:1094E000775A1836765AB74205D00B4F022300221E
:1094F00001268C377E52401CC0B2A842EDD32370A7
:10950000A273084A002180320F2002F092F909B0BC
:10951000F0BD0000F4130020C01200201815002038
:10952000F000002000D02724983A000024010020F9
:10953000C00D00203C010020F8B52E4C0546E06E21
:109540002D4A281A411E2067914215D21A21615EC8
:10955000081AFCF7A1F8294A294BFBF795FF0646A4
:1095600032200F46205EFCF797F832463B46FBF769
:10957000D9FEFCF7C7F86086002060761D481C23E2
:10958000C35E828C1F48008884461F4806881DE001
:109590006046484380181D4F80B23880302778439A
:1095A0006427643078431A4F6066C01985420BD235
:1095B000C8B2184932220880606EA25E411BC918E9
:1095C0008918A166E066F8BD491C6176617EB142EA
:1095D000DED33020424310486421101848430F491D
:1095E0004118E16660663221401B615EC018401878
:1095F000A066F8BD70000020CF0700009A999999E5
:109600009999B93F32010020240100204601002031
:1096100078ECFFFF3001002074270000C0BDF0FF90
:10962000FEB5294D2988491C8FB228492F800E8804
:10963000FCF732F8264A274BFBF726FF01910090F2
:1096400025483146FBF754FD244C218F4218B74280
:1096500006D3002028802248019E1018009D02E0B9
:109660001046019E009DFCF72BF833462A46FBF777
:1096700059FEFCF76BF8A086012580B2ED03A842E5
:1096800001D3401BA086E08BFCF71AF8154A164B55
:10969000FBF762FF0646A08E0F460090FCF710F81D
:1096A00032463B46FBF73EFEFCF750F880B2E086C0
:1096B000A84201D3401BE0860C4900980968486124
:1096C00000982087FEBD000030010020240100200A
:1096D0001904560E2D624040E17A0000700000200F
:1096E0001F050000F853E3A59B843E40541600205C
:1096F00070470000F8B531492F48086002F00EFAB3
:109700002F4800F0A3F92F4CE0822D48801C00F078
:109710009DF920832A48001D00F098F960832B48AA
:1097200029494180014640310979294F0906090E2E
:10973000617006D1C7800121C1870A2141870021BC
:109740008187244AC18E1170C18F2171818F61710F
:10975000817AA1708588052165626181C68830465D
:10976000FBF7C6FCA08101462846FBF7C1FC880038
:10977000081885B2164825816843FBF7A1FF164AF1
:10978000164BFBF7E9FEFBF7E1FFE081658231460E
:109790003846FBF7ADFC20820146C820FBF7A8FC49
:1097A000E0830120A083FCF7E5FCA082E2890C495C
:1097B0000C48FDF743FDF8BD45A6000868000020F1
:1097C000004F00081401002031020000C00D0020ED
:1097D000E803000018000020F853E3A59B843E40F6
:1097E000FF7F000054160020F8B5754C0027754E19
:1097F0002771012030807449C8200880207B401CDC
:109800002073C00706D0A08C411EA184022801D27B
:10981000C820A0840120C043FFF702FF0A2001F006
:1098200049FF7D20400101F05FFF02216748FDF7FD
:10983000D7FA00283FD00020654980000978664D9E
:1098400049000843634909780843A87210206872E8
:109850006248C1887D20C000FBF74AFC68736048FD
:109860005E490078A87328460B308A780270C97860
:1098700041705A49421C20310B7ED370497E1171D0
:109880005649D01C22310B7E5371497E9171534948
:1098900040310A7C0271497C41710022294617201F
:1098A00001F0F2FF0021172002F000F8022001F081
:1098B00051FF4C4D03E00120BEE7FEF75DFF0021A4
:1098C0000F2001F077FE28422064F6D0206C411C66
:1098D00073D040046FD58122D20100210F2001F006
:1098E000A8FF0021102001F065FE41063A48490E0C
:1098F0000022B430E16501F093FE374DB435687A4B
:10990000112858D102223849681DFBF75BFC00285A
:1099100051D1E81F027A69460A70407A4870A97AE4
:109920003180C820FBF7E4FB2749304E0880287BB4
:10993000A08428462838C08E3080294620482839FF
:10994000098F41842A48FDF775FC2085608C2949E0
:10995000FF30C33080B2608488420BD9494240183E
:10996000608430882349401C80B20B3130808842AB
:1099700000D3378030887D21C9004843618C40186E
:10998000606500F0A3F868460088E084A87C12496E
:109990006071C731420008460D466930FBF7EEFBA7
:1099A0006079294642001448FBF7E8FBA08CFF28A9
:1099B00001D001202070F8BDFFE700F049FF000052
:1099C000700000202401002032010020000400501B
:1099D000180100201901002034120020C00D0020C1
:1099E0001800002000D02724380100204401002066
:1099F00054160020E70300007C13002070B586B0E9
:109A000014216846FBF7D3FB01250F4EED0300221E
:109A100029463046FDF7F1F9012000240190029417
:109A20006946009503943046FDF71EF90320019026
:109A300002946946009503943046FDF715F902201B
:109A400001F0E6F806B070BD0004005000887047D1
:109A500070470000F8B5044600206A461080194D92
:109A600055222A70AA226A700322AA70661DEE701F
:109A70002A716971144A49008918AC712246E81D9F
:109A8000FBF77CFB002007E029186A4689781288DA
:109A900089186A461180401CB042F5DB611DA81C84
:109AA000FCF7A0F801466846018029190078C871C2
:109AB00068464078087221460931024800F0D8FB18
:109AC000F8BD000092150020C00D0020FEB5FFF784
:109AD00033FD2548FDF7AEFB244C86B22685607920
:109AE0000A21081AC000FBF7D7FD07460191A06EB6
:109AF000FBF7E6FD1E4A1F4BFBF72EFD00900D46BF
:109B00003046FBF7DDFD2B46009AFBF70BFC3A468F
:109B1000019BFBF707FCFBF719FE85B2A586E08BDE
:109B2000FBF7CEFD124A134BFBF716FD06460F4618
:109B30002846FBF7C5FD32463B46FBF7F3FBFBF738
:109B400005FE81B20120C003E186814201D3091ADA
:109B5000E186854201D3281AA0860349A08E0968B0
:109B600048612087FEBD00005416002070000020D0
:109B7000F853E3A59B843E40034A1168382389B219
:109B800099430143116070470030014010B5FDF763
:109B900041F910BD10B59AB034216846FBF707FBB8
:109BA00014210DA8FBF703FB1C2112A8FBF7FFFAF9
:109BB0001B4801680324E402A143C2148918016010
:109BC000FDF7B6FB17480169A1430161062000902B
:109BD000FF20013002900120039010200490022009
:109BE000099040040B90000100240C900A946846F0
:109BF000FDF7CCFD0F200D9003200E900F941094D4
:109C0000012111940DA8FDF797FC812012900320EB
:109C100080041890149412A8FDF7DCFB1AB010BD54
:109C20000070004040100240104801688215114346
:109C30000160C1680E4A1140C16001680D4A1140BF
:109C4000016081684908490081600168012292042D
:109C500091430160C168FD2212049143C16000215B
:109C60000161064904488860704700000010024006
:109C70000C40FF88F6FFF6FE0050000800ED00E003
:109C800070B5026801239B07114C124D984203D016
:109C9000A04201D0A84203D17026B2434E6832439D
:109CA000984203D0A04201D0A84204D103231B0252
:109CB0009A43CB681A4380239A430B691A43026084
:109CC0008A68C262096881620121416170BD000039
:109CD000000801400014014010B5CB06DB0E012145
:109CE000046A99408C430462016A9A4011430162FC
:109CF00010BD30B58468FF252D021B021343AC4311
:109D00000B432343836030BD826870239A430A4328
:109D100007210A438260704730B5026A5208520038
:109D20000262026A456883697024A3439C080B6839
:109D3000A40023430224A2438C684560144383613A
:109D400049684163046230BD30B5026A10239A430A
:109D50000262036A4568826973242402A2430C6884
:109D600024021443202293438A68456012011A4357
:109D7000846149688163026230BD30B5026AFF23A5
:109D800001339A430262026A4568C3697024A3439F
:109D90009C080B68A400234301246402A2438C683E
:109DA000456024021443C3614968C163046230BD45
:109DB00030B5026A01231B039A430262036A4568B5
:109DC000C26973242402A2430C68240214430122B2
:109DD000520393438A68456012031A43C461496879
:109DE0000164026230BD30B5036A046A640864002D
:109DF00004628469F025AC43120122430A24A34380
:109E00000B438261036230BD30B5036A1024A34363
:109E100003628469036A0F252D031203AC432243B6
:109E2000A024A343090119438261016230BD0000EF
:109E3000F8B5102405252D07AC62AF20800000F096
:109E4000EEFEAC6101F0CAFB2D4C2E4F2E4E60672A
:109E50000EE001F0C3FB6067FEF78EFC606C411CF6
:109E60006164142804D929A000F074FC2B48C76051
:109E7000606FB042EDD10026666420780127FF03B1
:109E8000030000F0A0FC04030B182C2E012239461D
:109E90002846FCF7B2FFFFF7A7FC06E0012239468F
:109EA0002846FCF7AAFFFBF7CDFE002239462846DC
:109EB000FCF7A3FF15E0A07B0122401CA0733946EC
:109EC0002846FCF79AFFFCF771F90022394628462C
:109ED000FCF793FFA07B052803D9267001E0FFF76C
:109EE00005F802210E48FCF77BFF002805D0002072
:109EF0000C49087001F058FAF8BD0120F8E700009D
:109F0000700000200400FA053001CADE44572049E1
:109F100044204552524F522E0D0A000000ED00E041
:109F2000000400504801002010B5818CC90707D0FB
:109F300001684A6801235B049A43836A1A434A60B2
:109F4000818C890707D501684A6801231B049A435D
:109F5000C36A1A434A60818C490707D501684A6879
:109F600001239B049A43036B1A434A60818C0907BF
:109F700007D501684A680123DB039A43436B1A4300
:109F80004A60818CC90607D50268916801231B03CA
:109F90009943836B19439160818C890607D50168C9
:109FA0008A6801235B039A43C36B1A438A60818CDE
:109FB000490612D503685A6801210905046C8A43D1
:109FC00022435A60026C8A4207D102685168032317
:109FD0005B059943436C19435160818C090607D591
:109FE00001684A680123DB04806C9A4302434A609B
:109FF00010BD0000F8B50446002680300660FCF76E
:10A0000003FF054620680068124F000709D50121AB
:10A010002B46002249052046009700F0A1FA0028AF
:10A020000DD12068006840070BD501212B46002286
:10A0300089052046009700F093FA002801D00320FC
:10A04000F8BD2020A067E0672666603426750020F2
:10A05000F8BD0000FFFFFF01F8B5154CC826E078F9
:10A06000002823D16079002820D101206071114D92
:10A07000686B0027002818D0686BC821081A0FE009
:10A080000D48E168405C61698847E068401CE06019
:10A09000E068C82800DBE760696BC820401A761EBC
:10A0A000E168814201D0002EEADC6771F8BD000052
:10A0B0005400002000000240F80C002070B5224C33
:10A0C000E07800283FD1207900283CD10120207180
:10A0D0001E4EF16900250906002933DA2156625720
:10A0E00091420AD1F06940062CD5A079002829D0E8
:10A0F000A5712089401C208124E0A179002903D189
:10A10000A0710A2000F08BFD00202056CC2148438E
:10A110000F494218206912181279B262401C0022BD
:10A120002061A256CC235A43895881420ADC25611A
:10A130002078401C207020780E2800D12570A0784F
:10A14000401CA070257170BD5400002000380140F3
:10A15000D001002010B5806A0022014640314A83B8
:10A160004A82FDF795FF10BD70B5846AA06FE56F58
:10A170002168896800260906002906DA212804D109
:10A1800052200653204600F06BF820688068400695
:10A1900006D5222D04D15A200653204600F047F858
:10A1A0002046803001681022114301602046FDF7EF
:10A1B0006FFF70BD10B501460968806A096889069D
:10A1C0001CD400225A210A5201680A68FF23013375
:10A1D0009A430A6001688A68520852008A600168DE
:10A1E0008A6840239A438A602021C167016E012951
:10A1F00004D101680A6810239A430A60016E01299C
:10A2000002D0FEF727F910BD5821095AFDF73EFF8D
:10A2100010BD10B5806A016E012902D0FEF71BF94E
:10A2200010BD5821095A4908FDF730FF10BD0168DB
:10A230000A68FF2321339A430A6001688A6852083A
:10A2400052008A60016E012904D101680A68102356
:10A250009A430A602021C167002101664166704768
:10A2600001680A68C0239A430A6020218167704709
:10A2700070B5164CE278002A0CD12279002A09D157
:10A280000122E2700025C82903DC0222A256002A1E
:10A2900001DCE57070BD0123E356CC2253430C4A28
:10A2A000D1500123E356CC2673439B180A4601463E
:10A2B000181DFAF763FF6078401C607060780E2804
:10A2C00000D16570A078401EA070E2E75400002025
:10A2D000D0010020F8B50446016880682369E6696A
:10A2E00018436369002533431843724A0B68724E62
:10A2F000334003430B602168486803231B039843E2
:10A30000E368184348602168A069914201D0236A3C
:10A3100018438B680B263602B34303438B606749AF
:10A32000236867488B420CD1C0688007800F06D035
:10A33000012839D0022835D0032821D11EE0012779
:10A340001FE060498B420AD1C0680C21084027D029
:10A35000042829D0082825D00C2811D10EE09342DA
:10A360000ED1C16803208002014019D00120800273
:10A37000091A19D0091A15D0814201D1082700E025
:10A3800010274F49504840398600934232D1002F60
:10A390000CD0022F0DD0042F10D0082F7FD126E033
:10A3A0000027EEE70227ECE70427EAE7FDF792F93A
:10A3B00006E00968C90605D4304603E0FDF7AAF9AE
:10A3C000002872D0626851005118814267D8110389
:10A3D000814264D3010E060250080023301859410F
:10A3E000FAF79CFE03210902411A384A55E0012080
:10A3F000C003E7E70122E369D20393422BD13B007C
:10A4000000F0E1F90906090C4D114D4D4D274D00A5
:10A41000FDF760F909E0FDF76DF906E00968C90686
:10A4200005D4304603E0FDF775F900283DD061689A
:10A4300040004A088018FAF75BFE80B20146244AC1
:10A44000103991422BD8511C01400007400F08439E
:10A4500029E01046EBE73B0000F0B5F90906090CCE
:10A460002112212121232100FDF734F90AE0FDF713
:10A4700041F907E00968C90606D4304604E00EE059
:10A48000FDF748F9002810D061684A081018FAF75B
:10A490002FFE80B201460E4A1039914203D90125A0
:10A4A00003E01046F0E72168C86000206066A066FF
:10A4B0002846F8BD00480040F369FFEF003801402E
:10A4C000401002400044004000093D00FFFC0F0026
:10A4D000EFFF0000F8B504464165403000262746EE
:10A4E000028380373E602220E0672546206F60357A
:10A4F00000281CD01749C162216F17480863216FDB
:10A5000016484863206F8663236F606D9C46134630
:10A510002168024660462431FCF7CEFA002806D0B6
:10A52000102038602E752020A0670120F8BD2E7500
:10A5300020680168FF2201321143016020688168B0
:10A5400001221143816020688168402211438160AB
:10A550000020F8BDB5A1000813A2000869A10008F9
:10A56000FFB581B005460F46044660350A9E39E0C6
:10A57000701C37D0FCF748FC0499401AB04222D82E
:10A58000002E20D02068016849072BD5C069C04340
:10A59000000527D401202168C002086220680168F4
:10A5A000FF22A13291430160206881684908490077
:10A5B00081602020A067E06780342060002028753B
:10A5C000032005B0F0BD20680168FF22A13291434D
:10A5D0000160206881684908490081602020A067E7
:10A5E000E067EBE72068C1693846884305D0002161
:10A5F00003988142BCD00020E3E70121F8E7000086
:10A6000010B504491020096808620248FDF742FDB0
:10A6100010BD00001C17002001490D2088707047F4
:10A620005400002010B5FEF71FFBFEF737FCC822D0
:10A6300002490348FDF7DEFE10BD0000F80C0020C3
:10A640001C170020F8B53E4C002321783D4A1D46DA
:10A65000082910D0072947D0062950D0052952D003
:10A66000042953D0032954D0002956D0012958D0A9
:10A6700002295AD05BE0A17800264A1F04E0314F3E
:10A68000BF5DFB189BB2761C9642F8DB6679277992
:10A690009A195118E3786278C9188918C9194018AD
:10A6A000C0430006000E1AD1012E14D0022E16D17E
:10A6B00025482449C018FAF761FD01F08BFF64209A
:10A6C00000F0A6FABFF34F8F21492048C860BFF3BE
:10A6D0004F8F00BFFDE759081046FFF7BBF9257003
:10A6E000E570A570A571F8BDA1795054491CC8B298
:10A6F000A071A178491F8842F5D1082001E060705F
:10A7000007202070F8BDE0700620FAE76071052090
:10A71000F7E7A070E5700420F3E7552807D1012082
:10A72000EFE7AA2803D10220EBE7032803D0257026
:10A73000E570A570F8BD032020702071F8BD000001
:10A740000B0100202E150020C00D00200400FA058A
:10A7500000ED00E010B5024A024900F0E5F910BD35
:10A7600011B90008600100202021020C01D0102145
:10A770001046020A01D010460839020901D01046DD
:10A78000091F820801D01046891E420801D0881E88
:10A790007047081A7047F8B5040C8BB2264682B28F
:10A7A0005E430D0C1046370C5843360480190021C7
:10A7B000794116466E43370C360480197941264696
:10A7C0006E438919F8BD30B47446641E2578641C44
:10A7D000AB4200D21D46635D5B00E31830BC1847F6
:10A7E0004900CA020243100000D004204A0D01D0E3
:10A7F00001221043044A490D914201D1022108432C
:10A80000012800D105207047FF0700008307FF22C1
:10A81000DB0E9A408907090E9940002808DB83085F
:10A8200009489B001B18186890430843186070473C
:10A830000007000F0838830804489B001B18D869DC
:10A8400090430843D861704700E400E000ED00E069
:10A85000BFF34F8F04490348C860BFF34F8F00BF59
:10A86000FDE700000400FA0500ED00E0F8B504463D
:10A870004F1EC8000838211815461E46086849684A
:10A880003A4606239A4310D02A463346FAF7FCFD8F
:10A890003A46D200083AA3181A687F1E5B68FAF796
:10A8A00041FD06223B469343EED1022F23D0042FD5
:10A8B00011D0062F2FD12A463346FAF7E5FDE36A79
:10A8C000A26AFAF72FFD2A463346FAF7DDFD636ADE
:10A8D000226AFAF727FD2A463346FAF7D5FDE369DF
:10A8E000A269FAF71FFD2A463346FAF7CDFD6369E0
:10A8F0002269FAF717FD2A463346FAF7C5FDE368E1
:10A90000A268FAF70FFD2A463346FAF7BDFD6368E1
:10A910002268FAF707FDF8BD002210B5134610466D
:10A920000149FAF719FE10BD0000F03F10B5FAF723
:10A93000F9FC10BD002210B5134610461146FAF777
:10A940000BFE10BD10B50721024A00200907FAF7D7
:10A950007BFE10BD01030000034A10B50020110763
:10A96000FAF772FE10BD000001FDFFFF02E008C80B
:10A97000121F08C1002AFAD170477047002001E079
:10A9800001C1121F002AFBD1704700000149086075
:10A99000704700006401002008B50021684601707E
:10A9A0006B46012202212C2000F052FF0221684652
:10A9B00001706B4601222C2000F04AFF08BD000008
:10A9C00038B504466D20694608706B460122074978
:10A9D0002E2000F03DFF0649002C01D0054A00E082
:10A9E000054A2E2000F01AFF38BD000006080000BE
:10A9F00006180000070600000716000038B50446D8
:10AA00006B4602220021362000F0EEFDB321230028
:10AA1000FFF7D9FE0E0F08153A3A3A3A1C273A3A90
:10AA20002F34483A002168460170407841084900B7
:10AA300014E06946087880088000401C04E06946FC
:10AA4000087880088000801C08701DE06846027845
:10AA50000A404832027041788020014368464170C4
:10AA600012E0684602780A40027040784106490EBA
:10AA7000F4E7694648780221084303E069464878CC
:10AA8000FD210840694648706B46012200213620AE
:10AA900000F0DEFE012200AB11463620013300F04B
:10AAA000D7FE38BD69460878CF2108406946203076
:10AAB000CAE708B5032168464170012101706B4661
:10AAC00002220021362000F0C3FE0122D20306211B
:10AAD0002D2000F0A3FE012000F09AF80120FFF7DE
:10AAE0008DFF08BD08B5020A69464A7008706B46BA
:10AAF000022204212D2000F0ABFE032069460870DD
:10AB00006B46012206212D2000F0A2FE002069469E
:10AB100008706B46012206212D2000F099FE0A21C3
:10AB20002D2000F047FD08BDF8B516460F46044637
:10AB3000002503E03946B047641C6D1C20780028CE
:10AB4000F8D12846F8BD0000F8B54A002B4B520D4D
:10AB5000D6182B4A0C460546142E2BDA002E12DA94
:10AB6000284BFAF7DFFB00221346FAF735FE40D2F6
:10AB7000002C03DA0124E40700253AE020462843AC
:10AB800037D0214C14E0214F0B46F7403B402B437C
:10AB900031D01C4BFAF7C6FB00221346FAF71CFE15
:10ABA00027D2002C03DD01200005F0400419BC432E
:10ABB00000251EE0332E1EDC33460027143BFF43E6
:10ABC000DF40384217D00F4BFAF756FC00221346ED
:10ABD000FAF702FE0DD2002C0ADD142E0CD0342020
:10ABE000811B012088404019A84200D2641C054600
:10ABF000BD4321462846F8BD641CF9E701FCFFFF70
:10AC00009C7500883CE4377E0000F03FFFFF0F009A
:10AC10007D2110B5C900484300F001F810BD0021A6
:10AC200040E000BF00BF00BF00BF00BF00BF00BFCB
:10AC300000BF00BF00BF00BF00BF00BF00BF00BF1C
:10AC400000BF00BF00BF00BF00BF00BF00BF00BF0C
:10AC500000BF00BF00BF00BF00BF00BF00BF00BFFC
:10AC600000BF00BF00BF00BF00BF00BF00BF00BFEC
:10AC700000BF00BF00BF00BF00BF00BF00BF00BFDC
:10AC800000BF00BF00BF00BF00BF00BF00BF00BFCC
:10AC900000BF00BF00BF00BF00BF00BF00BF00BFBC
:10ACA00000BF491C8142BCD37047FFB581B01E462E
:10ACB0000F46040026D00B9903980143A06A39433C
:10ACC000826807209047002818DB0A99A06A314360
:10ACD000826806209047002810DB25462035A97998
:10ACE000032F01D908200143032E01D90420014379
:10ACF000A06A826809209047002806DA0120C04334
:10AD000005B0F0BD0020C043FAE7384600F000F976
:10AD10002060304600F0FCF860600A986870039884
:10AD2000A870EF702E710B9868710020E8E70000A2
:10AD3000F7B50446002090B000900190002C05D09B
:10AD40006A46062101F080FC062803DA0020C04391
:10AD500013B0F0BD684640780102684600780004F0
:10AD60000918684680780818FAF7AAFC054668466C
:10AD70000391007901026846C0780004091868460A
:10AD800040790818FAF79CFC032206460F46920702
:10AD90005C4BFAF721FD07D200225B4B3046394667
:10ADA000FAF764FB06460F4603229207554B2846E6
:10ADB0000399FAF711FD07D20022534B2846039955
:10ADC000FAF754FB054603912068FAF779FC02462E
:10ADD0000B4630463946FAF7BFFB07460A20079173
:10ADE000205EFAF759FC3A46079BFAF74DFB0646F8
:10ADF00008200991205EFAF73DFC0021C943FAF7CB
:10AE000085FAFAF7C1FC3246099BFAF78BFA0691EC
:10AE100008906068FAF754FC02460B4628460399EE
:10AE2000FAF79AFB05461A200E46205EFAF734FC24
:10AE30002A463346FAF728FB0C9009911620205E2B
:10AE4000FAF72AFC099B0C9AFAF76CFA05910A901A
:10AE50002A46334638460799FAF716FB059B0A9AA5
:10AE6000FAF712FB05910A901420205EFAF714FC01
:10AE70003A46079BFAF708FB07461C200791205E1D
:10AE8000FAF70AFC2A463346FAF7FEFA0E900B91BF
:10AE90001820205EFAF700FC0B9B0E9AFAF742FA94
:10AEA0002A463346FAF7F0FA0B910E902069FAF72A
:10AEB000F3FB0B9B0E9AFAF735FA2A463346FAF75C
:10AEC000E3FA05460E46E068FAF7E6FB2A46334603
:10AED000FAF728FA3A46079BFAF724FA059B0A9AEA
:10AEE000FAF720FA01229207084BFAF7CDFA024648
:10AEF0000B46129C0898069903C411980CC00020B8
:10AF000026E70000FFFF5F4100007041E17A843FC7
:10AF100000B50121C9040300FFF755FC081A050814
:10AF20000B0E1114171A0320C00400BD0720C00423
:10AF300000BD0F20C00400BD1F20400300BD3F2006
:10AF4000400300BD7F20400300BDFF20400300BD43
:10AF5000084600BDFEB5264F0D4604000FD0002D5B
:10AF60000DD0264600202036B071F07129680D20E2
:10AF70008847002801DA7800FEBD102801D0384645
:10AF8000FEBDA562E968002901D028208847204637
:10AF900000F030F80028F3DBA06AA52182680E20BB
:10AFA0009047A06A962182680F209047A06A0221EC
:10AFB000826862209047A06A002182680E20904734
:10AFC000A06A002182680F2090477179302001919A
:10AFD00000900623202201212046FFF766FE00286C
:10AFE000CEDB204600F0AEF80028C9DB0020FEBD15
:10AFF000FFFFFFFF10B586B0044614216846FAF73C
:10B00000D6F8002C7ED0A06A122143686A46102030
:10B010009847122877D168460078012201016846D6
:10B02000407812030009081843492081884201DD55
:10B03000801A20816846837840780007000D181830
:10B040006081884201DD801A6081684600790122B2
:10B0500001016846C0781205000309186846407966
:10B06000000908183549E060884201DD801AE06077
:10B07000684640790007030B6846807900021B1878
:10B080006846C07918182061884201DD801A206165
:10B090006846417A007A0002081802B22848012165
:10B0A0000904A282824201DD521AA2826A46D37A40
:10B0B000927A12029A1812B2E282824201DD521A88
:10B0C000E2826A46537B127B12029A1812B22283E2
:10B0D000824201DD521A22836A46D37B927B12029E
:10B0E0009A1812B26283824201DD521A62836A4662
:10B0F000537C127C12029A1812B2A283824204DD9F
:10B10000501A01E00BE008E0A083A06A0168282043
:10B110008847002806DA0120C04306B010BD002091
:10B12000C043FAE7C011C0072034002800D08020B7
:10B1300060710020F1E70000FF070000FFFF07003B
:10B14000FF7F000010B5040009D0A06A07218268C3
:10B1500008209047002805DA0120C04310BD0020D8
:10B16000C04310BD072020342070002010BD000017
:10B17000FEB50446002001900090607973494000BC
:10B180000E5A61782578491E7148CFB20163042DAB
:10B1900077D0072D75D000210291217801736C4979
:10B1A000E379012292058969002B6CD0914381617A
:10B1B0006748217A4173217A82698907890B0A439A
:10B1C00082610021042000F034FB324661492E20C8
:10B1D00000F024FB3846FFF7F3FB5F4E0522705D5D
:10B1E000810040185D49431807212B2000F030FBF7
:10B1F0005B49029801220B180B21282000F028FB44
:10B20000705D584980000A580C21282000F011FB7D
:10B21000E079554980004018A1794900425A02213D
:10B22000272000F0FBFA51487E00825B0421272092
:10B2300000F0F4FAE079002829D0A07804282CD076
:10B2400028206946087220220621272000F0E6FA0D
:10B2500002AB01222621272000F0FAFA44493801E6
:10B260004018E178890042580821272000F0E1FACF
:10B27000A17A601C627A0902114313D016E000E043
:10B2800001E0012188E71143F608816190E764221B
:10B290000621272000F0C2FAE0E710206946087274
:10B2A0000246D1E733490172090A4172417A007AB4
:10B2B0000A0202432021272000F0B0FA2E4F0C2171
:10B2C00023203A6800F0B5FAF0198288042123207F
:10B2D00000F0A4FAA07900280BD0E07927490122D8
:10B2E00043180021212000F0B3FA0320019001202F
:10B2F00000902A07120F1001024360780021800796
:10B30000000B0243019800050243009840040243E9
:10B310002079C006400902436079C00602431F201D
:10B3200000F087FAA07861780123084302040848F6
:10B33000DB030261E179490319430A4302610021F9
:10B34000082000F076FA0020FEBD00007CC700084F
:10B35000940100200428000024C7000824000020D5
:10B36000420000202CC700084CC7000858C700083E
:10B370005CC700084110000044C7000844000020DA
:10B3800038B50C4607498A8B002102432C2000F077
:10B3900045FA684604706B46012206212C2000F015
:10B3A00057FA38BD9401002010B5FFF7F5FA10BD2B
:10B3B00010B504460421362000F0FCF80121C90232
:10B3C000002C01D0084300E08843024604213620C7
:10B3D00000F02FFA10BD000038B540206946087013
:10B3E00000210E2000F0E6F80446002211460E204F
:10B3F00000F01FFA6B46012200210D2000F028FA10
:10B40000074A00210F2000F014FA00F0EDF922465F
:10B4100000210E2000F00DFA02480021017338BD12
:10B42000F8FF2724B4010020FEB505460420694634
:10B430000870514C0020607521462031206348710E
:10B440000873A0836063A06300F0C8F84B4E2060CF
:10B4500002E000F0C3F82060B042FAD10020FFF70C
:10B46000CDFA00F0BBF8464E20603078242801D990
:10B47000243806E00621F9F73BFE0622101A4001A7
:10B480000843020601040A4301020A430243B26070
:10B49000706000211E2000F0CCF900F09FF82060C1
:10B4A0006B4601220021242000F0D2F91E20FFF774
:10B4B00019FB86B2300AA0730420FFF713FB07467E
:10B4C00000F08CF820603806000E0DD0022069468E
:10B4D000087101AB012212212D2000F0B9F9A08BD7
:10B4E000012109030843A08300F078F820600620BA
:10B4F000FFF7F8FA60600720FFF7F4FAA060F006A3
:10B50000C00E207501D110202075C0B200F0DCF90A
:10B51000E80707D0FFF7CDFAA08B0121C902084345
:10B52000A0830AE00521362000F02EF815490840D6
:10B5300002460521362000F071F90120FFF75EFA7E
:10B540000021042000F036F8A0610021262000F040
:10B5500031F815218903084302460021262000F016
:10B5600068F900222621362000F058F900F036F85C
:10B5700020600020FEBD0000940100203001CADEE2
:10B5800018000020FFFD000038B5094C89B280B2D8
:10B590006B46022200F028F8002806D16846407861
:10B5A000010268460078081884B2204638BD0000C1
:10B5B000FFFF000038B50024E44389B280B26B4637
:10B5C000042200F011F8002806D103216846435CEC
:10B5D0002202D418491EFAD5204638BD10B50021E4
:10B5E0000846FFF7E7FF10BD38B5002909D0402411
:10B5F00020436C462070C8B27F2906D860700220B4
:10B600000AE069460870012006E0802420436C4669
:10B610006070C809A0700320694600F0B5FF38BD0E
:10B6200010B5144603460A4621461120FFF7DCFFF9
:10B6300010BD10B50346052200211520FFF7D4FFE9
:10B6400010BD10B50346052200211720FFF7CCFFDF
:10B6500010BD38B5054600206946087000F0C4F8F2
:10B66000FF2401342246002D01D0032212020021C2
:10B670000D2000F0D3F8002D13D06B4601220321DA
:10B680000F20FFF7B1FF68460078000709D5FFF7E4
:10B69000A3FE224600210D2000F0C0F80020C04388
:10B6A00038BD002038BD10B5024601210A2000F047
:10B6B000C0F810BD10B5044600211A20FFF77AFF2C
:10B6C000000D22030005120B024300211A2000F096
:10B6D000B0F810BD10B5024602492E2000F09EF8C9
:10B6E00010BD000004180000F8B505466B460122A5
:10B6F00003210420FFF778FF0126114C3607002DA7
:10B700000DD02A4600210C2000F088F86946087800
:10B710001021084369460870A069304307E0694674
:10B720000878EF21084069460870A069B0430B46CD
:10B73000A06101220321042000F08AF8F8BD000076
:10B740009401002010B502460021182000F066F890
:10B7500010BD0000F8B50746002568460570B8071B
:10B76000204C2E4600280ADA8020694608706B4675
:10B77000012200210D2000F06BF801202073F80752
:10B780006946087821D006210843694608706B464F
:10B79000012200210D2000F05BF803210F20FFF7AC
:10B7A000F3FE8121C900084219D040206946087083
:10B7B0006B46012200210D2000F04AF80020FFF71F
:10B7C000F7FD00252673ED4309E002210843694691
:10B7D00008706B46012200210D2000F039F8284640
:10B7E000F8BD0000B40100201CB56B460122032106
:10B7F0000F20FFF7F9FE684600784022C10910408B
:10B80000C9014000814208D0012069460871024602
:10B8100001AB03210D2000F01BF81CBD08B56B46E1
:10B820001A70120A5A7089B280B2022200F010F81F
:10B8300008BD38B500236C46E254120A5B1C042B89
:10B84000FADB89B280B22346042200F001F838BD49
:10B8500038B58024002909D0C02528436D462870BA
:10B86000C8B27F2907D86870022009E020436946E2
:10B870000870012004E020436870C809A870032004
:10B88000694600F02BFF38BD10B51446012312188D
:10B890009B029A4202D90020C04310BD0B46821E73
:10B8A00021460920FFF7D4FF002010BD10B5054A3E
:10B8B0008905126901430A4300210820FFF7B9FFF7
:10B8C000002010BD9401002038B504466B460122CB
:10B8D0000E212B20FFF788FE68460078E10640091C
:10B8E0004001C90E0143684601706B4601220E21DA
:10B8F0002B20FFF7ADFF38BD10B5002142541C06C8
:10B90000120A22431B0A491C0429F7DB10BD000060
:10B9100013B501231A4669460248FCF79DFD0098BD
:10B920001CBD00001C1700207CB50024254668467D
:10B93000FFF77FFE04206946220E2D0215432202E6
:10B940000C5C1443401EF7D5204629467CBD7CB5CF
:10B95000002425466846FFF774FE04206946220E3F
:10B960002D02154322020C5C1443401EF7D52046DD
:10B9700029467CBDFBF756FAFEF70CF9FDF788F96E
:10B980003F494048002522C005608561C5613E49A8
:10B990000562C1600838FBF7D7FBFDF765F9FDF7D5
:10B9A0007DFAFDF719FAFDF72BF90524012224078A
:10B9B000D1032046FBF721FAFDF79CFEFDF708F8BE
:10B9C000FAF7ECF8FAF794FAFAF762FAFCF7C6FD20
:10B9D0000721A015FFF7D4FCFFF7E6FC01221103B5
:10B9E0002046FBF70AFA2748C8222849C830FCF746
:10B9F00001FDFCF79BFF264F264E274C3878002888
:10BA00000FD13078002801D003280AD10121C902C2
:10BA10002248FBF7E5F9002803D101210846FBF78E
:10BA2000A7FCE078002828D06078002825D0E570B1
:10BA300072B620780F280AD90120184900038861BE
:10BA4000FEF7F6F901201549000388620CE0012297
:10BA500051031248FBF7D1F9FEF7EAF90121002260
:10BA600049030E48FBF7C9F962B6FCF785FE208C46
:10BA70000028C3D0401E2084C0E7FCF77DFEBDE750
:10BA8000007C004054160020FFFF0000F80C00204E
:10BA90005A000020850000201401002000040050FE
:10BAA00010B586B01848FBF7D2FA14216846F9F7AA
:10BAB0007EFB164800900320019000200290052094
:10BAC00069460007FBF7D0F869461148FBF7CCF848
:10BAD00069461048FBF7C8F8FCF728FF0121084623
:10BAE000FBF746FCFF2401342046FBF719FC0A490A
:10BAF00008680422104308602046FBF721FCFBF78E
:10BB000027FC06B010BD000054160020FFFF000007
:10BB100000040050000800500070004010B50122E1
:10BB2000920217491748FAF767FA1548164902882A
:10BB30008A4223D0018004218180FF21F531C18018
:10BB40000A21018100211E224181D24382810122EA
:10BB5000C28181834323C3860223038778234387DB
:10BB60008287C28702464032118451849184C18306
:10BB7000918014238382118200F02CFD10BD0000FF
:10BB8000C00D002000FC0008AA550000F0B51FB44D
:10BB900096B084460C460246199D189803904900B9
:10BBA00068006300490840080193002A01D001267B
:10BBB00000E000269E19FE4BF6185B109E422BD328
:10BBC0006E00039F0296002F00D00127F719F84E50
:10BBD000F84BBE199E421FD3039E0346F64F3343D4
:10BBE00009D03B469C4201D1002A04D0019B002A87
:10BBF00005D0012604E0002039461BB0F0BD002628
:10BC00009E19EE4B9E4207D8039F029E002F00D044
:10BC10000127F6199E4207D92B4660462146189AFD
:10BC2000FEF784FE1BB0F0BD0023002C29DAE44EA1
:10BC3000B04226DAE34EB04201DB022321E0DE4EC1
:10BC4000B0421EDBE04E070DBE19142E09DD34276D
:10BC5000BF1B039EFE400196BE40039FBE420BD019
:10BC60000FE0039F002F0CD11427BF1B0646FE4098
:10BC70000196BE40864204D1019BDE07F60F0223E7
:10BC80009B1B0E46164318D1002D16DA002C03D04C
:10BC9000022B01D0012B06D00220FEF777FEFEF723
:10BCA0003BFE1BB0F0BD0220FEF770FEFEF734FE37
:10BCB0000122D20751401BB0F0BD039E002E61D17E
:10BCC000BF4EB04220D1C148844201D1002A08D0E1
:10BCD000B948814209DB002D10DB189829461BB0BA
:10BCE000F0BD0020B4491BB0F0BD002D06DA0122E2
:10BCF0002946D207189851401BB0F0BDB449794489
:10BD0000086849681BB0F0BDAB4FB84225D1002D83
:10BD10001FDA002904D0B14212D1002A09D018E05C
:10BD2000002A72D1A649E20F0020D20711431BB0AE
:10BD3000F0BD0020E20F0146D20711431BB0F0BD59
:10BD4000B14206DA234600203946F9F705FC1BB05C
:10BD5000F0BD104621461BB0F0BDB14212DA0126FB
:10BD6000B607B54203D1234610461946FEE3994E65
:10BD7000B54207D1261E05DB1046314600F040FCD7
:10BD80001BB0F0BD67007F081646002A40D100298D
:10BD90000AD08B4A914229D1002C0EDD002D1CDBEC
:10BDA000002011461BB0F0BD022B16D0002C14D081
:10BDB000012B12D1002C14DB0FE0002C28DA002D0F
:10BDC00009DB012B03D000207D491BB0F0BD002012
:10BDD00081491BB0F0BD012B03D0002001461BB0F0
:10BDE000F0BD00200121C9071BB0F0BD724A91428D
:10BDF0000ED1002C01DA002B17D0022B06D0002028
:10BE0000C043F9F749FC1BB0F0BD90E20120F8E710
:10BE1000E217521C94461A4307D000220892664C3F
:10BE200062465B1E1A4307D009E00120FEF7AEFD13
:10BE3000FEF780FD1BB0F0BD0022644C0892674AFB
:10BE400090427DDD664B674A98421FDD914202DCDD
:10BE5000002D05DB4DE05848814217DB002D48DD01
:10BE60000220FEF793FDFEF76DFD05460E4600220B
:10BE7000534B21460898F9F707FB0846710049081B
:10BE8000C00FC007014328461BB0F0BD914215DA30
:10BE9000002D2EDA0220FEF779FDFEF753FD054650
:10BEA0000E460022464B21460898F9F7EDFA72003B
:10BEB0005208C80FC0070243114617E03E4B994293
:10BEC00023DD002D15DD0220FEF760FDFEF73AFDB3
:10BED00005460E4600223A4B21460898F9F7D4FA57
:10BEE000084671004908C00FC007014328461BB02F
:10BEF000F0BD0220FEF74AFDFEF72EFD490049087D
:10BF0000E20FD20711431BB0F0BD00223046394684
:10BF1000F9F7ACFA012205460E46D243F9F794FB35
:10BF2000314A324BF9F7A8FA2A463346F9F7ACFA08
:10BF30000022284BF9F7A0FA07462A46334600E0CC
:10BF400064E0039110461946F9F79EFA3A46039BBE
:10BF5000F9F79AFA0746032209915207244B28461B
:10BF60003146F9F791FA07910C90224A204B384656
:10BF70000999F9F789FA074601911F4A1F4B28468C
:10BF80003146F9F781FA3A46019BF9F76FFA07460D
:10BF90000B460246099107990C98F9F7C3F9002559
:10BFA0000E462846079B0C9AF9F760FA3A4627E0B6
:10BFB000FFFF1F00FFFF0F000000F03F0000E0FF49
:10BFC0000000F07F0000404301FCFFFF0000F0BFD5
:10BFD000560B00000000E03F0000F0FF0000E041D1
:10BFE0000000F043FFFFEF3F555555555555D53FE0
:10BFF0004715F73FFE822B6544DF5DF80BAE543EDC
:10C00000099BF9F739FA02460B4652E10125002057
:10C010002D05A94207DA352230463946F9F714FBD7
:10C0200006463420C0430A151218FE481018039023
:10C030000803FD49000B01430F46FC49884201DC1F
:10C04000002003E0FA49884202DA0120119005E05D
:10C05000002011900398401C7F1B039011980597B6
:10C06000C200F4480F927844801843680268394649
:10C0700030460D930292F9F7F9F907910C9030468A
:10C080000D9B029A0599F9F74DF902460B460020DF
:10C09000E549F9F761FA09910490079B0C9AF9F7C1
:10C0A000F3F9129000201090E3480D4678440068A0
:10C0B0000E90012178104907084311990D9B8904BE
:10C0C00040180121C90447183946029A0E98F9F719
:10C0D000CDF93246059BF9F7CFF902460B462946C2
:10C0E0001098F9F7D1F9064602913B4629460E9A77
:10C0F0001098F9F7C9F9079B0C9AF9F7BDF9324680
:10C10000029BF9F7B3F9099B049AF9F7BDF9059178
:10C11000129A0A902B4610461946F9F7B5F90646C9
:10C120000246C6480F460B4606217844FEF79EFBA2
:10C1300032463B460091049010461946F9F7A4F99F
:10C14000009B049AF9F7A0F906460F462B461946BC
:10C15000129A1098F9F7E6F8059B0A9AF9F794F9FC
:10C1600032463B46F9F7DEF8109A079104902B46C9
:10C1700010461946F9F788F9B14E00223346099165
:10C180000290F9F7CFF8079B049AF9F7CBF8002053
:10C190000746024633460091F9F768F9099B029A6F
:10C1A000F9F764F9079B049AF9F766F906460D91C9
:10C1B0003A462946009B1098F9F766F907910C90CA
:10C1C0002B463046129A0D99F9F75EF905460E4650
:10C1D0003A46009B05990A98F9F756F933462A46DC
:10C1E000F9F7A0F802460B460746099107990C9803
:10C1F000F9F798F800250E462846079B0C9AF9F7A0
:10C2000035F93A46099BF9F737F9074607220991AC
:10C2100052078C4B31462846F9F736F907910090C2
:10C22000894A884B38460999F9F72EF90746019152
:10C23000864A874B31462846F9F726F93A46019B4C
:10C24000F9F770F8834B7B440F9A9B181A685B6868
:10C25000F9F768F8029009910398F9F71DFA05912A
:10C260000490099B029A07990098F9F75BF87A4BBA
:10C270007B440F9A9B181A685B6817460393F9F77B
:10C2800051F8059B049AF9F74DF80E462846059B90
:10C29000049AF9F7EBF83A46039BF9F7E7F8079B9E
:10C2A000009AF9F7E3F8099B029AF9F7E5F80246D4
:10C2B0000B46199900200C900F461898F9F7E4F8EE
:10C2C000029104903B460C9A19991898F9F7CEF808
:10C2D0002A463346F9F7D8F8029B049AF9F722F870
:10C2E00009910E902A46334639460C98F9F7CCF856
:10C2F00006460F46099B0E9AF9F714F8574A0D4661
:10C30000914220DB5242AA18024310D132463B46EA
:10C31000F9F7ACF804900391514A524B09990E98E1
:10C32000F9F700F8039B049AF9F756FA1ED2022097
:10C33000FEF72CFBFEF706FB49004908E20FD20787
:10C3400011431BB0F0BD6A00474B52089A420DD30F
:10C35000464AAA18024300D0CBE532463B46F9F7DD
:10C3600085F8099B0E9AF9F737FAF5D9680000238A
:10C3700040082C490393020D3D4B5218984223DD8F
:10C3800001200005521CD04042195000400D4018B9
:10C3900038497944096813468C463749C1408B4374
:10C3A00012030121120B090551181422101AC14061
:10C3B0000391002D01DA4842039062463046394627
:10C3C000F9F754F806460F4632463B4609990E984F
:10C3D000F8F7A8FF00252A46284B28460591F9F7CB
:10C3E00053F807910C90264A264B28460599F9F7F1
:10C3F0004BF80091029032463B4628460599F9F7E2
:10C4000035F8099B0E9AF9F737F81F4A1F4BF9F7D1
:10C410003BF8009B029AF8F785FF07460B46024659
:10C42000099135E001FCFFFF0000F03F8E9803000A
:10C430007AB60B0066070000A8070000D2060000CD
:10C440000000084009C7EE3FFD033ADCF5015B142C
:10C45000E02F3EBEA60500006C05000000009040E5
:10C46000FE822B654715973C00CC904000346F3F0F
:10C470000000E03FC2040000FFFF0F00432EE63F34
:10C48000396CA80C615C20BEEF39FAFE422EE63F03
:10C4900007990C98F8F746FF05460E46079B0C9A3D
:10C4A000F8F7E4FF3A46099BF8F7E6FF09912A46B8
:10C4B00033460E9010461946F8F7E6FF0746024647
:10C4C0002F480B46059105217844FEF7CFF93A46EF
:10C4D000059BF8F7D9FF2A463346F8F7CDFF074604
:10C4E000019128463146099B0E9AF8F7CDFF099B2A
:10C4F0000E9AF8F717FF012304910C9000229B0776
:10C5000038460199F8F7B2FF05910E903A46284651
:10C510003146019BF8F7B8FF059B0E9AF9F71CF816
:10C52000049B0C9AF8F7A2FF2A463346F8F79EFFC1
:10C530000022144BF8F7A0FF064603980D460005AD
:10C5400041190915002912DC30462946039AF9F7EA
:10C550007BF8FEF745F9042801D1FEF7FDF93046D6
:10C560002946039AF9F770F8064601E004E0291815
:10C570000B46324621460898F8F786FF1BB0F0BDFF
:10C58000640300000000F03FF0B58C460025102643
:10C59000052109078E620E4C08E067467F5DE76063
:10C5A000A768FF07FCD0E7681F706D1C8542F4DBAD
:10C5B0000020074606E0E760A568ED07FCD0E568C7
:10C5C0001D54401C9042F6D38E610020F0BD000047
:10C5D0000030014070B572B60124074DA402214617
:10C5E0002846F9F7EFFC002804D0224603492846E4
:10C5F000F9F78CFD62B670BD00FC0008C00D00208C
:10C60000F8B506460C46F9F7F5F9051E0F4600D0B9
:10C610000120014349000B484908411AC90F0DD0B8
:10C62000002E01D0012100E000210C4361004908E7
:10C63000401AC00F02D10120FEF7A8F9284639465A
:10C64000F8BD00000000F07FF8B515460E4607461D
:10C65000002407E03819C0B200F008F8641C287004
:10C66000E4B26D1CB442F5D33046F8BD10B50446B3
:10C67000FCF71EF8EE20FBF7EEFFFCF752F8204621
:10C68000FBF7E9FFFCF74DF8FCF712F8EF20FBF79A
:10C69000E2FFFCF746F80020FBF7B0FF0446FCF78A
:10C6A00022F8204610BD704770B50D460446FBF7D2
:10C6B000FFFFEE20FBF7CFFFFCF733F82046FBF738
:10C6C000CAFFFCF72EF82846FBF7C5FFFCF729F850
:10C6D000FCF709F80A20FEF7A2FA70BDF0B50025B4
:10C6E000102605279C463F070B46BE620C4C06E011
:10C6F000595DE160A168C907FCD0E1686D1C854205
:10C70000F6DB002007E06146095CE160A168C9072B
:10C71000FCD0E168401C9042F5D3BE610020F0BD22
:10C72000003001400000010203040005405C0000ED
:10C73000A05C0400C06C0800805C0400E03F1E00A8
:10C74000E07D1E0007A9022570889B880A0016005C
:10C75000010006000100020087008D002D001A3143
:10C7600052001A339A001A351D011A376B003B31FB
:10C77000BE003B335E013B3596023B3700009959C2
:10C780009959EB518F421E45142E0080EB51F5282C
:10C790003333E13A703DE13AC235852BC23533334C
:10C7A000C235C235AE47E13A5138A33051380000A6
:10C7B000000000000000010203040607080903044A
:10C7C00006080C10182030000000000102030400CD
:10C7D000000000000000F03F000000000000F83FF3
:10C7E00000000000000000000000004003B8E23F2D
:10C7F000000000000000000006D0CF43EBFD4C3EDF
:10C80000033333333333E33FFFAB6FDBB66DDB3FD3
:10C810004D268F515555D53F01411DA96074D13F1B
:10C8200065DBC9934A86CD3FEF4E454A287ECA3F15
:10C830003E5555555555C53F93BDBE166CC166BF97
:10C840002CDE25AF6A56113FF16BD2C541BDBBBE90
:10C85000D0A4BE726937663E0000000000000000F0
:10C8600080C800080000002068010000BC5A0008D1
:10C87000C4C8000868010020E01A00007CA9000874
:10C880000124130704380D091E0805400826091065
:10C890004008560A131D043B08BE0516D8BC4010BC
:10C8A000085201033AC842077052030CE5800C1B82
:10C8B0000202DD14090102628149C8013A2940924D
:04C8C00004922000BE
:04000005080050C1DE
:00000001FF
